S02B0000433A2F576F726B2F736F6674776172652F4F70656E424C542F5461726765742F44656D6F2F41524DEF
S315080000003C20002017020008D1220008D12200084F
S31508000010D1220008D1220008D1220008D1220008E6
S31508000020D1220008D1220008D1220008D1220008D6
S31508000030D1220008D1220008D1220008D1220008C6
S31508000040D1220008D1220008D1220008D1220008B6
S31508000050D1220008D1220008D1220008D1220008A6
S31508000060D1220008D1220008D1220008D122000896
S31508000070D1220008D1220008D1220008D122000886
S31508000080D1220008D1220008D1220008D122000876
S31508000090D1220008D1220008D1220008D122000866
S315080000A0D1220008D1220008D1220008D122000856
S315080000B0D1220008D1220008D1220008D122000846
S315080000C0D1220008D1220008D1220008D122000836
S315080000D0D1220008D1220008D1220008D122000826
S315080000E0D1220008D1220008D1220008D122000816
S315080000F0D1220008D1220008D1220008D122000806
S31508000100D1220008D1220008D1220008D1220008F5
S31508000110D1220008D1220008D1220008D1220008E5
S31508000120D1220008D1220008D1220008D1220008D5
S31508000130D1220008D1220008D1220008D1220008C5
S31508000140D1220008D1220008D1220008D1220008B5
S31508000150D1220008D1220008D1220008D1220008A5
S31508000160D1220008D1220008D1220008D122000895
S31508000170D1220008D1220008D1220008D122000885
S30D08000180D1220008D122000873
S3150800018872B64D484D4901604D49072291438D463F
S315080001984C484D494D4A00F07DF84D484D494E4A60
S315080001A800F078F84D484E494E4A00F073F84E4824
S315080001B84E494F4A00F06EF84E484F494F4A00F0EC
S315080001C869F84F484F49504A00F064F84F48504973
S315080001D8002200F06AF84F484F49091A082903DB34
S315080001E8002202600430016040484149884205D02F
S315080001F80268043003B4904703BCF7E70020864634
S31508000208EC4602F009FE00200021444A904772B6DF
S315080002182B49072291438D462A482B492B4A00F039
S3150800022839F82B482B492C4A00F034F82B482C4926
S315080002382C4A00F02FF82C482C492D4A00F02AF8A9
S315080002482C482D492D4A00F025F82D482D492E4AC7
S3150800025800F020F82D482E49002200F026F82D48EF
S315080002682D49091A082903DB0022026004300160B7
S315080002781E481F49884205D00268043003B49047CF
S3150800028803BCF7E700208646EC4600200021234AEF
S315080002989047FEE7884207D0521A05D003780130FE
S315080002A80B700131013AF9D17047884202D00270C1
S315080002B80130FAE77047000008ED00E00000000882
S315080002C83C200020F86F00080000002018000020D5
S315080002D828030008280300088C660008F86F000839
S315080002E800000020000000208C6600088C660008C4
S315080002F88C6600088C6600088C6600088C66000800
S315080003088C6600088C660008F86F0008180000203C
S315080003183C1000203C1000203C180020452200080C
S3150800032808B54FF43053C4F20103586B10F0450F63
S3150800033807D14FF43052C4F20102506B10F0450F42
S31508000348FBD010F0040F06D04FF0040001F01EFE93
S315080003584FF0030008BD10F0010F06D04FF001005A
S3150800036801F014FE4FF0010008BD40F2FF5001F0FD
S315080003780DFE4FF0000008BD10B504464FF4305383
S31508000388C4F20103586B10F0450F07D14FF43052E9
S31508000398C4F20102506B10F0450FFBD010F0040FA1
S315080003A806D04FF0040001F0F1FD4FF0030010BD30
S315080003B810F0010F06D04FF0010001F0E7FD4FF0ED
S315080003C8010010BD01F09AFDA0424AD140F2FF5043
S315080003D801F0DCFD4FF0000001F098FD4EF208012F
S315080003E8CFF6FF51014000293ED000283FDB10F028
S315080003F8804F3FD110F0005F3FD110F0805F3FD1AA
S3150800040810F0006F3FD110F0806F3FD110F0807F59
S315080004183FD110F4000F3FD110F4800F3FD110F4EC
S31508000428001F3FD110F4801F3FD110F4002F3FD191
S3150800043810F4802F3FD110F4003F3FD110F4803FCD
S315080004483FD110F4004F3FD110F4804F3FD110F43C
S31508000458005F3FD100F00803002B14BF1A200020C4
S3150800046810BD4FF0100010BD4FF0000010BD4FF042
S315080004781C0010BD4FF0090010BD4FF00A0010BD52
S315080004884FF00B0010BD4FF00C0010BD4FF00D00DB
S3150800049810BD4FF00E0010BD4FF00F0010BD4FF005
S315080004A8100010BD4FF0110010BD4FF0120010BD1E
S315080004B84FF0130010BD4FF0140010BD4FF0150093
S315080004C810BD4FF0160010BD4FF0170010BD4FF0C5
S315080004D8180010BD4FF0190010BD00BF2DE9F041F6
S315080004E882B004464FF0000001F010FD10F0007FBE
S315080004F840F042814FF000020092019240F2D00388
S315080005081846C2F200004FF0080101604FF01005C6
S3150800051845604FF040038360C2604FF48062026111
S3150800052801F0D4FC2846FFF727FF0146002840F0CB
S315080005382B8140F2D000C2F2000040F27401C2F2E8
S3150800054800010B6803FA05F303604FF037054560A9
S315080005584FF0400282604FF00001C1604FF480639B
S31508000568036101F0B3FC2846FFF706FF0146002899
S3150800057840F00A8140F21C00C2F200004FF0FF3535
S3150800058805604FF0080646604FF0300282604FF06B
S315080005980201C1604FF0000505614FF00103436190
S315080005A801F0C2FC40F2D000C2F2000005604FF02C
S315080005B8330646604FF040028260C5604FF480619A
S315080005C8016101F083FC3046FFF7D6FE0146002894
S315080005D840F0DA80ADF104084FF43055C4F201054D
S315080005E840F22A664FF4001707E0384601F0C4FCC3
S315080005F818B101F0B1FC48F8040F6B6B3342F4D01C
S315080006084FF0080001F0B8FC30B14FF0080001F0CF
S31508000618BDFC4FF00401B7E04FF0020001F0ACFC56
S3150800062830B14FF0020001F0B1FC4FF00201ABE027
S315080006384FF0200001F0A0FC30B14FF0200001F087
S31508000648A5FC4FF006019FE04FF4007001F094FCFA
S3150800065830B14FF4007001F099FC4FF0070193E0B0
S3150800066840F2FF5001F092FC00984FEA006242EA15
S31508000678106300F47F4143EA012300F47F0043EA4C
S315080006881022012C3DD112F4802F78D040F2D004E4
S315080006982046C2F2000040F27403C2F200031A6848
S315080006A84FEA024101604FF0370444604FF04003B7
S315080006B883604FF00002C2604FF48061016101F067
S315080006C805FC2046FFF758FE014600285CD140F293
S315080006D8D000C2F200004FF0020404604FF006048E
S315080006E844604FF0400383604FF00002C2604FF445
S315080006F88061016101F0EAFB2046FFF73DFE0146ED
S3150800070842E012F4803F3DD040F2D0042046C2F2BF
S31508000718000040F27403C2F200031A684FEA024165
S3150800072801604FF0370444604FF0400383604FF090
S315080007380002C2604FF48061016101F0C7FB2046E0
S31508000748FFF71AFE0146F8B940F2D000C2F20000D7
S315080007584FF0000303604FF0060444604FF0400270
S315080007688260C3604FF48061016101F0AFFB2046E7
S31508000778FFF702FE014607E04FF00E0104E04FF0CE
S31508000788250101E04FF02501084602B0BDE8F081D1
S3150800079800B583B04FF001038DF807304FF40060B9
S315080007A8C4F202004FF4006101F090FA18B94FF04C
S315080007B800008DF807009DF8070003B000BD00BFCC
S315080007C82DE9F04782B04FF000048DF8074040F253
S315080007D85C00C2F200004FF07603037504604460BB
S315080007E88460C460046101F043FB4FF0030001F024
S315080007F85FFB4FF0010001F055FB40F2D000C2F252
S315080008080000046044608460C4604FF4806101613C
S3150800081801F05CFB4FF480354FF0800609E005F1DE
S31508000828FF34251E304601F0A7FB002800F02B816F
S3150800083804E0304601F0A0FB0028F0D04DB140F2A4
S31508000848FF5001F0A3FB4FF0000004E04FF003004F
S3150800085801E04FF003008DF807009DF8072012B154
S315080008689DF8070008E140F2D000C2F200004FF4F4
S31508000878D57404604FF0080545604FF0400383605F
S315080008884FF00001C1604FF48062026101F01EFB5F
S315080008984FF43050C4F20100436B13F0450F14D1DE
S315080008A84FF480314FF43054C4F2010401F1FF3596
S315080008B82946636B13F0450F06D105F1FF31636BC3
S315080008C813F0450F00F0DB8011B113F0040F06D0C2
S315080008D84FF0040001F05AFB4FF003020BE013F047
S315080008E8400F06D04FF0400001F050FB4FF00002D1
S315080008F801E04FF000028DF807209DF8070048B977
S3150800090840F24405C2F200054FF001022A604FF092
S31508000918804518E040F2D0042046C2F200004FF0A5
S31508000928000505604FF0370444604FF040018160C8
S31508000938C5604FF48063036101F0C8FA2046FFF7E3
S315080009481BFD8DF8070040F2D000C2F200004FF0F8
S31508000958000303604FF0370444604FF0400181609C
S31508000968C3604FF48062026101F0B0FA2046FFF7CF
S3150800097803FD8DF807009DF8070000287AD14FF087
S31508000988000740F2D004C2F20004B846B94645F05A
S31508000998004646F4801A4FF43055C4F20105C4F8E7
S315080009A800904FF0370666604FF04003A360C4F81E
S315080009B80C904FF480612161204601F087FA304691
S315080009C8FFF7DAFC8DF807009DF8072012B19DF8A5
S315080009D8070051E0C4F800A04FF0290060604FF006
S315080009E84003A360C4F80C804FF480612161204657
S315080009F801F06CFA6A6B12F0450F03D16A6B12F0B4
S31508000A08450FFBD012F0040F06D04FF0040001F092
S31508000A18BDFA4FF0030004E040F2FF5001F0B6FAC1
S31508000A2840468DF807009DF8073013B19DF8070072
S31508000A3822E0404601F06AFA07F10107002804DBBC
S31508000A484FF6FF739F42AAD103E04FF6FE718F4215
S31508000A5806D94FF01B018DF807109DF807000BE023
S31508000A6810F0804F06D040F24400C2F200004FF062
S31508000A78020202609DF8070002B0BDE8F087002967
S31508000A887FF414AF24E7651E7FF4D3AEDEE600BF15
S31508000A9838B501F013FA002800F0D78040F244036D
S31508000AA8C2F200031868042800F0D28040F2D00089
S31508000AB8C2F200004FF0000101604FF002024260E6
S31508000AC84FF0C0048460C1604FF48063036101F08D
S31508000AD8FDF9FFF725FC0446002840F0C48001F01C
S31508000AE815FA40F24805C2F2000528604FF00400DE
S31508000AF801F00CFA68604FF0080001F007FAA860E0
S31508000B084FF00C0001F002FAE86040F24400C2F225
S31508000B1800000168012903D9062901D0022956D1FE
S31508000B2840F2D000C2F200004FF0000101604FF019
S31508000B38030242604FF040038360C1604FF480614E
S31508000B48016101F0C3F94FF43050C4F20100436B58
S31508000B5813F0450F07D14FF43052C4F20102536B14
S31508000B6813F0450FFBD013F0040F06D04FF004001E
S31508000B7801F00CFA4FF0030475E013F0010F06D0E4
S31508000B884FF0010001F002FA4FF001046BE001F0A2
S31508000B98B5F9032818BF102465D140F2FF5001F0B3
S31508000BA8F5F94FF0000001F0B1F910F4604F02D1E1
S31508000BB84FEA10430DE010F4005F4CD110F4804F53
S31508000BC84CD110F4004F4CD14FF0010301E04FF01F
S31508000BD8010340F24401C2F200010868042842D021
S31508000BE840F27404C2F20004236040F2D000C2F254
S31508000BF800004FEA034202604FF0090343604FF0D2
S31508000C08C00181604FF00004C4604FF4806202613D
S31508000C1801F05CF9FFF784FB044620BB01F076F97E
S31508000C2840F23405C2F2000528604FF0040001F0CE
S31508000C386DF968604FF0080001F068F9A8604FF090
S31508000C480C0001F063F9E8600DE04FF025040AE0AE
S31508000C584FF0000407E04FF0130404E04FF01004C7
S31508000C6801E04FF00F04204638BD00BF70B40146B6
S31508000C7840F24403C2F200031C6880F8564040F26A
S31508000C887400C2F200000268A1F8542040F2340643
S31508000C98C2F2000633684FEA13604FEA90150D70E2
S31508000CA8C0F383024A7000F003008870C3F307454F
S31508000CB8CD70C3F307220A71DBB24B7176684FEA27
S31508000CC816604FEA0015CD80C6F30742CB8898B25E
S31508000CD840EA1215CD8002F00F020A72C6F30723FE
S31508000CE8D8B24FEAD0154D72C3F380128A72C3F38D
S31508000CF84015CD72C3F300120A734FF000054D7301
S31508000D08012C48D803F003004FEA80230B610D69CC
S31508000D18F2B245EA82040C6140F23406C2F20006D1
S31508000D28B0684FEA10630D6945EA93120A61C3F37E
S31508000D38C2040C7503F007064E75C0F307434FEA5D
S31508000D4853158D75C3F38202CA7503F003044FEA77
S31508000D5844060E76C0F307200B7E43EAD0150D76B7
S31508000D680E690A7E0C7A4FF0010303FA04F40C653F
S31508000D7802F1020203FA02F24FEAE275A2FB042321
S31508000D8804FB053306F10106A2FB064506FB0355D7
S31508000D98C1E912452CE0022C2AD106F03F044FEA95
S31508000DA804460E6140F23400C2F2000085680B69F9
S31508000DB84FEA156243EA02240C610E69C5F3074037
S31508000DC840EA06030B61C5F307200D694FF00102D7
S31508000DD84FF00004561944F100034FEAC34545EAA3
S31508000DE85632CA644FEAC6448C644FF400760E65D8
S31508000DF8C0F380164E7600F03F004FEA40048C7622
S31508000E0840F23405C2F20005AA688B7EC2F3C01602
S31508000E1843EA0600887602F07F04CC76ED684FEA46
S31508000E2815624FEAD2130B77C2F341164E77C2F30F
S31508000E388200887702F003044FEA8402CA77C5F36A
S31508000E480743CE7F46EA9310C877C3F3401481F860
S31508000E5820404FF0000081F8210003F0010281F8D4
S31508000E682220C5F307234FEAD31681F82360C3F374
S31508000E78801481F82440C3F3401281F82520C3F36F
S31508000E88001681F82660C3F3810481F8274003F029
S31508000E98030381F82830C5F3460581F829504FF031
S31508000EA8010481F82A4040F24803C2F200031A688E
S31508000EB84FEA126681F82C60C2F307454FEA052601
S31508000EC8CE85CD8DADB2C2F307263543CD854FEA1B
S31508000ED802620A635A680D6B4FEA126645EA0645C6
S31508000EE80D630D6BC2F3074645EA06250D630D6BC0
S31508000EF8C2F3072635430D63D2B281F834209A68BF
S31508000F084FEA126681F83560C2F307454FEA056667
S31508000F188E638D6BC2F3072645EA06458D638D6B8E
S31508000F28D2B245EA02258D63DB688A6B42EA136505
S31508000F388D63C3F3074291F83C5045EA121581F8C8
S31508000F483C5002F00F024FEA0225CD87CA8F92B2AB
S31508000F58C3F307252A43CA87C3F3460381F84030F3
S31508000F6881F8414070BC704710B540F24403C2F29C
S31508000F7800031968032933D0022934D8B0F5805FED
S31508000F8834D0B0F5006F16D14FF00100FFF7A6FA76
S31508000F98044668BB40F25C00C2F200004FF000034A
S31508000FA803750360436083604FF40061C1600361A1
S31508000FB800F05EFF1CE04FF00000FFF78FFA0446CA
S31508000FC8B0B940F25C00C2F200004FF000020275A8
S31508000FD8026042608260C260026100F049FF07E071
S31508000FE84FF0270404E04FF0000401E04FF027040F
S31508000FF8204610BD10B540F2D003C2F200031860AF
S315080010084FF007045C604FF040029A604FF000000A
S31508001018D8604FF480611961184600F057FF2046DA
S31508001028FFF7AAF910BD00BF2DE9F04184B04FF0CB
S3150800103800068DF80F604FF00C004FF0010100F024
S31508001048D3FE4FF40064C4F2020420464FF00801A8
S315080010584FF00C0200F040FE20464FF009014FF011
S315080010680C0200F039FE20464FF00A014FF00C0238
S3150800107800F032FE20464FF00B014FF00C0200F04C
S315080010882BFE20464FF00C010A4600F025FE4FF4C9
S315080010984067C4F2020738464FF002014FF00C02C7
S315080010A800F01AFE4FF4706301934FF001058DF8AE
S315080010B809504FF002088DF808808DF80A608DF8F7
S315080010C80B50204601A900F051FD4FF0040101918B
S315080010D83846694400F04AFD4FF4805001908DF86F
S315080010E80B60204601A900F041FD4FF400670197FF
S315080010F88DF808808DF80B60204601A900F036FDAA
S315080011083846294600F082FE4FF48000294600F04A
S315080011186BFE00F09FFEFFF753FB8DF80F009DF856
S315080011280F2012B19DF80F003BE0FFF7B1FC8DF8D0
S315080011380F009DF80F3013B19DF80F0031E040F20B
S315080011485C00C2F200004FF00001017501604160C1
S315080011588160C160016100F08BFE40F27800C2F23E
S315080011680000FFF783FD8DF80F009DF80F0068B99A
S3150800117840F27802C2F20002B2F854304FEA03404D
S315080011884FF00001FFF736FF8DF80F009DF80F1096
S3150800119829B94FF40060FFF7E7FE8DF80F009DF8B0
S315080011A80F0004B0BDE8F0812DE9F8430746164656
S315080011B8BDF820204FF0000140F21800C2F20000E6
S315080011C8017040F25804C2F20004216040F2E405B6
S315080011D8C2F2000529604FF43050C4F20100C1621A
S315080011E840F24401C2F200010C68022C05D14FEA0C
S315080011F8562646EAC3564FF40072914640F2D00086
S31508001208C2F2000002604FF0100343604FF0400539
S3150800121885604FF00001C1604FF48064046100F0F6
S3150800122855FE4FF480344FF0800508E004F1FF348A
S31508001238284600F0A1FE002800F0CB8004E02846E6
S3150800124800F09AFE0028F1D04FF01000FFF794F846
S315080012588046002840F0AA8040F21C00C2F200002E
S315080012684FF0FF320260C0F804904FF09003836095
S315080012784FF00205C5604FF0000505614FF0010102
S31508001288416100F051FE40F2D000C2F2000006604B
S315080012984FF0110444604FF040028260C5604FF475
S315080012A88063036100F012FE2046FFF765F8804662
S315080012B800287BD13C464FF43055C4F2010540F26C
S315080012C82A664FF400471DE0384600F055FEC8B1B7
S315080012D800F042FE206000F03FFE606000F03CFE31
S315080012E8A06000F039FEE06000F036FE206100F0EC
S315080012F833FE606100F030FEA06100F02DFEE0616B
S3150800130804F12004696B3142DED04FF0080000F082
S3150800131833FE30B14FF0080000F038FE4FF00408ED
S3150800132844E04FF0020000F027FE30B14FF002000B
S3150800133800F02CFE4FF0020838E04FF0200000F0CD
S315080013481BFE30B14FF0200000F020FE4FF00608D3
S315080013582CE04FF4007000F00FFE90B14FF40070C7
S3150800136800F014FE4FF0070820E000F0F5FD2546CA
S3150800137845F8040B07F1FF37304600F0FDFDC0B904
S3150800138809E04FF0FF374FF40016304600F0F4FD39
S3150800139808B1002FE9D140F2FF5000F0F7FD40F2FE
S315080013A80000C2F200004FF0000202604046BDE8A5
S315080013B8F88300F0D1FD6060304600F0DDFD0028B6
S315080013C8E9D000F0C9FD686005F10804A7F102072D
S315080013D8DBE7013C7FF433AF36E700BF2DE9F04F72
S315080013E885B082461646BDF838404FF0000140F2EF
S315080013F81802C2F20002117040F25800C2F2000048
S31508001408016040F2E405C2F2000529604FF4305243
S31508001418C4F20102D16240F24401C2F2000108682E
S31508001428022805D14FEA562646EAC3564FF40074F1
S31508001438254640F2D0031846C2F2000004604FF071
S31508001448100444604FF0400282604FF00001C1600A
S315080014584FF48063036100F039FD2046FEF78CFFE0
S315080014688346002840F0D38040F2D000C2F200003C
S3150800147806604FF0180444604FF0400282604FF04F
S315080014880001C1604FF48063036100F01FFD204628
S31508001498FEF772FF8346002840F0B98040F21C0028
S315080014A8C2F200004FF0FF37076045604FF090061C
S315080014B886604FF00004C46004614FF0010242617F
S315080014C800F032FD02944FF43056C4F2010640F299
S315080014D81A674FF4804960E0484600F04DFD002839
S315080014E85BD0029AC2F500701F2830D8830801938A
S315080014F853D055464FF000046FEA0400019A811844
S3150800150801F001030393DAF8000000F02DFD04F159
S3150800151801040AF10408019884427CD10FE0454683
S3150800152855F8040B00F020FDD8F8040000F01CFD5F
S3150800153804F1020405F10408019B9C42EFD10198C5
S315080015480AEB800A029A02EB8001029125E0DAF892
S31508001558000000F009FDDAF8040000F005FDDAF8E5
S31508001568080000F001FDDAF80C0000F0FDFCDAF8D6
S31508001578100000F0F9FCDAF8140000F0F5FCDAF8C7
S31508001588180000F0F1FCDAF81C0000F0EDFC0AF18E
S31508001598200A029901F120010291706B38429BD00A
S315080015A84FF0080000F0E8FC30B14FF0080000F0F2
S315080015B8EDFC4FF0040B2AE04FF0020000F0DCFCCB
S315080015C830B14FF0020000F0E1FC4FF0020B1EE0CC
S315080015D84FF0100000F0D0FC30B14FF0100000F0CA
S315080015E8D5FC4FF0050B12E04FF4007000F0C4FC70
S315080015F830B14FF4007000F0C9FC4FF0070B06E055
S3150800160840F20001C2F200014FF000030B60584691
S3150800161805B0BDE8F08F039A002A80D0DAF80400EE
S3150800162800F0A2FC04F1010408F1040801998C42AF
S315080016387FF475AF83E700BF38B5054618B340F29F
S31508001648D0031846C2F2000040F27402C2F2000241
S3150800165811684FEA014404604FF00D0444604FF0E6
S31508001668400383604FF00002C2604FF48061016155
S3150800167800F02CFC2046FEF77FFE044628B900F049
S3150800168845FC286001E04FF02604204638BD00BF17
S3150800169800B583B04FF000030193FFF779F80128E6
S315080016A818BFFF2009D101A8FFF7C6FF18B9019886
S315080016B8C0F3432001E04FF0FF0003B000BD00BFB0
S315080016C808B5FFF7E5FF042804D0FF2814BF012052
S315080016D8022008BD4FF0000008BD00BF00B597B04E
S315080016E8FFF7A2FC68B940F20400C2F200000178CC
S315080016F801F0FE0303706846FFF7B8FA4FF00000DA
S3150800170808E040F20403C2F200034FF001021A701F
S315080017184FF0030017B000BD08B540F20403C2F243
S3150800172800034FF001021A7050B9FFF7C9FF38B91C
S3150800173840F20400C2F20000017801F0FE030370CB
S3150800174840F20402C2F20002107808BD2DE9B0433F
S31508001758ADF5027D88461746C8B120E04FF0000966
S315080017684FF40075E219009502A84FEA42224B4643
S31508001778FFF71AFDB0B9FFF7A3FF0128FBD008EB5E
S31508001788442002A92A4604F037FF8CB90DE003F174
S31508001798FF34E4B2002BE1D14FF001000CE04FF022
S315080017A8010009E04FF0010006E04FF0000003E0F1
S315080017B804F1FF30C4B2D5E70DF5027DBDE8B08364
S315080017C82DE9F043ADF5037D0F469046E8B124E0D0
S315080017D84FF400754FF0000902A807EB44212A4682
S315080017E804F00AFF04EB0802009502A84FEA422211
S315080017F84B46FFF7F3FD064608B1052810D1FFF753
S315080018085FFF0128FBD08CB90DE003F1FF34E4B281
S31508001818002BDDD14FF001000CE04FF0010009E084
S315080018284FF0010006E04FF0000003E004F1FF3036
S31508001838C4B2D1E70DF5037DBDE8F08310B596B0BF
S31508001848144640F20403C2F200031A7812F0010F94
S3150800185821D1032922D8DFE801F0020513194FF030
S31508001868000023E0E8B96846FFF700FA129B4FEA3A
S315080018785322139942EAC15020604FF0000015E040
S315080018884FF4007020804FF000000FE060B94FF069
S31508001898200121600AE04FF0030007E04FF004003A
S315080018A804E04FF0000001E04FF0000016B010BD4C
S315080018B84FF00000C4F2AA20704700BF82B04FF468
S315080018C86053C4F202031A6842F0010018604FF028
S315080018D800029A60196821F0847020F48031196032
S315080018E843F21000C2F200405860196821F48020BB
S315080018F81860DA60009201921A6842F48031196019
S315080019084FF46050C4F20200036803F400320192EF
S31508001918009901F101010091019B1BB9009AB2F5E2
S31508001928A06FF1D14FF46050C4F20200016811F4B7
S31508001938003F14BF012100210191019B012B46D1CB
S315080019484FF46050C4F20200026C42F08051016400
S315080019584FF4E043C4F200031A6842F440411960A0
S3150800196883688360826842F400418160836843F42F
S31508001978A052826045F20C41C0F24071416003688A
S3150800198843F0807202604FF46050C4F202000168A6
S3150800199811F0007FFBD04FF47053C4F2020340F2F3
S315080019A805621A604FF46050C4F20200816821F09B
S315080019B803038360826842F0020181604FF4605035
S315080019C8C4F20200836803F00C02082AFAD14FF41D
S315080019D86D41CEF200014FF00060886002B0704792
S315080019E84FF47053C4F20203186900280DDA4FF44D
S315080019F87051C4F2020140F22312C4F267524A60D7
S31508001A0848F6AB13CCF6EF534B6070474FF4705358
S31508001A18C4F202031A6942F000401861704700BF11
S31508001A284FF47053C4F20203D86070474FF47053EA
S31508001A38C4F20203D86810F4803F1BD14FF47051E2
S31508001A48C4F20201CA6812F0100F16D14FF4705387
S31508001A58C4F20203D86810F0EF0F11D14FF4705191
S31508001A68C4F20201CA6802F00203002B0CBF082060
S31508001A78072070474FF0010070474FF00500704780
S31508001A884FF00600704700BF00B583B04FF0080353
S31508001A988DF80730FFF7CAFF8DF807009DF807008D
S31508001AA8012807D1FFF7C2FF8DF807009DF8071030
S31508001AB80129F7D09DF8070003B000BD70B50546A3
S31508001AC80E46FFF7E1FF082816D14FF47054C4F202
S31508001AD80204236923F440702061216941F40072E5
S31508001AE82261236943F0010020612E60FFF7CCFFCD
S31508001AF8216921F00102226170BD00BF70B5054653
S31508001B0841B1012909D0022914BF4FF440764FF490
S31508001B18007604E04FF0000601E04FF48076FFF700
S31508001B28B3FF082821D14FF47054C4F2020420697F
S31508001B3820F440712161226916432661236923F03E
S31508001B48F8002061216941F00202154325612369DD
S31508001B5843F480302061FFF797FF216921F00202DC
S31508001B682261236923F0F801216170BD2DE9F0018E
S31508001B784FF000034FF001054FF0030705FA03F28B
S31508001B880C68144094423DD106684FEA430207FAA6
S31508001B9802F46FEA040426400660066891F804C051
S31508001BA80CFA02FC4CEA060606600E7906F1FF36C0
S31508001BB8F6B2012E17D886683440846086684C7950
S31508001BC804FA02F43443846046689CB205FA04FCB5
S31508001BD826EA0C064660466891F806C00CFA04F42C
S31508001BE8A4B234434460C6689CB24FEA440407FA70
S31508001BF804F426EA0406C660C468CE7906FA02F230
S31508001C082243C26003F101031C4605FA03F20E6873
S31508001C181640964253D102E0BDE8F0017047D0F865
S31508001C2800804FEA430207FA02F66FEA060606EA52
S31508001C38080CC0F800C0D0F8008091F804C00CFA67
S31508001C4802FC4CEA080CC0F800C091F804C00CF174
S31508001C58FF3C5FFA8CFCBCF1010F0FD9C668A4B229
S31508001C684FEA440407FA04F426EA0406C660C46878
S31508001C78CE7906FA02F22243C26020E0D0F808803C
S31508001C8806EA08068660866891F805C00CFA02F81E
S31508001C9848EA06068660D0F804C09EB205FA06F831
S31508001CA82CEA080CC0F804C0D0F804C091F80680DD
S31508001CB808FA06F6B6B246EA0C064660CEE703F117
S31508001CC80103102B7FF45AAFA6E700BF0369194230
S31508001CD80CBF00200120704730B401F007034FEA13
S31508001CE883034FEAD10101F1080150F821504FF05A
S31508001CF80F0404FA03F425EA040440F8214050F8CE
S31508001D08214002FA03F2144340F8214030BC7047D8
S31508001D1810B44FF46053C4F20203996801F00C0238
S31508001D28042A09D0082A0DD0002A38D14FF41053AE
S31508001D38C0F2F403036037E04FF4D853C0F2B70390
S31508001D48036031E04FF46051C4F202014C684A68F6
S31508001D5802F03F0114F4800F4FF46053C4F20203F3
S31508001D685A68C2F3881319BF4FF4D854C0F2B70497
S31508001D784FF41054C0F2F404B4FBF1F404FB03F175
S31508001D884FF46052C4F202025368C3F3014404F1E3
S31508001D9801044FEA4402B1FBF2F1016004E04FF492
S31508001DA81054C0F2F40404604FF46053C4F20203FA
S31508001DB89C68C4F3031240F20801C2F200018C5C65
S31508001DC8026822FA04F242609C68C4F382240C5D15
S31508001DD822FA04F484609B68C3F34233C95C22FA86
S31508001DE801F2C26010BC704739B14FF46051C4F2B1
S31508001DF802010B6B1843086370474FF46053C4F22B
S31508001E0802031A6B22EA00001863704739B14FF4C7
S31508001E186051C4F202014B6C1843486470474FF48A
S31508001E286053C4F202035A6C22EA000058647047E9
S31508001E3839B14FF46051C4F202014B6A184348623B
S31508001E4870474FF46053C4F202035A6A22EA000044
S31508001E585862704708B54FF400604FF00101FFF764
S31508001E68E7FF4FF400604FF00001FFF7E1FF08BDF8
S31508001E7810B44FF43053C4F201035C6841688268B1
S31508001E881143C26811430268114302690A4324F4DC
S31508001E98FD4424F07F042243007D02435A6010BCA7
S31508001EA8704700BF48F2A003C4F22523186070479C
S31508001EB84FF43053C4F20103186070474FF4305397
S31508001EC8C4F20103186800F00300704710B40268EA
S31508001ED84FF43053C4F201039A60DC6824F4FF61B6
S31508001EE821F00704826841681143C26811430069F2
S31508001EF801432143D96010BC704700BF4FF43053E3
S31508001F08C4F201031869C0B2704700BF82B04FF027
S31508001F180003019342F61441C4F2010140180190E6
S31508001F28019A106802B0704710B402684FF430532B
S31508001F38C4F201035A6241689962DC6A24F0F7041C
S31508001F48C268816811430269114340690143214304
S31508001F58D96210BC704700BF4FF43053C4F201036E
S31508001F68D3F88000704700BF4FF43053C4F201031A
S31508001F78C3F88000704700BF4FF43053C4F201031A
S31508001F88596B08420CBF0020012070474FF43053A4
S31508001F98C4F201039863704730B585B004460D4608
S31508001FA8038A23F440504FEA00414FEA1143EA886E
S31508001FB813432382A08920F4B05121F00C034FEA79
S31508001FC803424FEA12402989AB8841EA0302698924
S31508001FD80A4393B21843A081A28A22F440714FEAB1
S31508001FE801434FEA1340AA891043A0826846FFF7BF
S31508001FF88FFE4FF48051C4F201018C4205D04FF48C
S31508002008A053C4F201039C4201D1039800E0029848
S31508002018A28911B2002909DA00EB800101EB8100D7
S315080020282B684FEA4305B0FBF5F208E000EB80039E
S3150800203803EB83002D684FEA8502B0FBF2F248F2FB
S315080020481F51C5F2EB11A1FB02104FEA50134FEAD4
S3150800205803154FF0640103FB1122A08903B2002B74
S315080020680DDA4FEAC20202F1320248F21F51C5F2EE
S31508002078EB11A1FB0220C0F342132B430CE04FEAF5
S31508002088021202F1320248F21F51C5F2EB11A1FB06
S315080020980220C0F343132B439BB2238105B030BDFE
S315080020A829B181898AB242F40053838170478389AA
S315080020B823F400514FEA01424FEA124383817047DD
S315080020C84FEAC1514FEAD1528280704780884FEA59
S315080020D8C0514FEAD1507047038819420CBF0020F7
S315080020E80120704700B589B04FF0000300930193AB
S315080020F802930393049305930693079346F28C6019
S31508002108C0F60000694604F017F940B9009848B1C6
S315080021189DF8081081F01002C2F3001004E04FF091
S31508002128000001E04FF0000009B000BD46F28C60DF
S31508002138C0F60000704700BF08B540F2E800C2F2D2
S3150800214800004FF0000380F8243246F2AC61C0F66E
S3150800215800014FF00A0203F0F3FC38B940F2E80030
S31508002168C2F200004FF0010280F8242208BD00BF21
S3150800217838B540F2E803C2F2000393F824020128AE
S3150800218805D140F2E800C2F2000003F0EBFF4FF475
S31508002198A054C4F201044FF0400520462946FFF72B
S315080021A89BFF0028F9D046F28C60C0F6000004F0C0
S315080021B8EBF838BD08B540F2E803C2F2000393F815
S315080021C82402012805D140F2E800C2F2000003F013
S315080021D8C9FF08BD70B5064640F2E803C2F2000317
S315080021E893F82402012812D1304640F2E801C2F2D7
S315080021F8000104F07FF9002809DA40F2E800C2F283
S3150800220800004FF0000180F8241203F0ABFF317884
S3150800221891B14FF4A054C4F201044FF0800520464A
S31508002228FFF74EFF20462946FFF756FF0028F9D044
S3150800223816F8011F0029F2D170BD00BF00B583B09A
S3150800224872B6FFF73BFB4FF020004FF00101FFF78E
S31508002258DDFD4FF004004FF00101FFF7C5FD4FF40F
S315080022680064C4F2020420464FF006014FF0080243
S31508002278FFF732FD20464FF007014FF00802FFF737
S315080022882BFD4FF000038DF806304FF001008DF84E
S3150800229807004FF002058DF804504FF040010091F1
S315080022A88DF8055020466946FFF760FC8DF80450FE
S315080022B84FF08002009220466946FFF757FC00F067
S315080022C85DFD00F069FDFCE708B546F2BC60C0F69E
S315080022D800004FF03D0100F009FD08BD08B500F003
S315080022E891FB80B100F08EFD00F09AFB4EF608537C
S315080022F8CEF200034FF400421A6048F20400C0F612
S3150800230800000168884708BDF8B5044602F1FF379A
S31508002318BFB2F2B100F10103DF190E1A6FEA000025
S31508002328391801F00105A25D04F8012B00F082FDB9
S31508002338BC420FD1F8BDA05D254605F8010B00F093
S3150800234879FDA95D617005F1010400F073FDBC42D1
S31508002358F1D1F8BD002DEED0A35D04F8013B00F0DD
S3150800236869FDBC42E7D1F8BD08B5FDF750FF08BDC1
S3150800237810B5044600F05EFD47F6FF73C0F6000385
S315080023889C4205D94BF6FF70C0F6000084427DD9F9
S3150800239800F050FD4BF6FF71C0F600018C4205D9D6
S315080023A84FF6FF72C0F60002944272D900F042FD59
S315080023B84FF6FF73C0F600039C4205D94FF6FF7027
S315080023C8C0F60100844267D900F034FD4FF6FF7164
S315080023D8C0F601018C4205D94FF6FF72C0F6030212
S315080023E894425CD900F026FD4FF6FF73C0F6030346
S315080023F89C4205D94FF6FF70C0F60500844251D9AC
S3150800240800F018FD4FF6FF71C0F605018C4205D994
S315080024184FF6FF72C0F60702944246D900F00AFD45
S315080024284FF6FF73C0F607039C4205D94FF6FF70AF
S31508002438C0F6090084423BD900F0FCFC4FF6FF7150
S31508002448C0F609018C4205D94FF6FF72C0F60B0291
S31508002458944230D900F0EEFC4FF6FF73C0F60B0332
S315080024689C4205D94FF6FF70C0F60D00844225D95F
S3150800247800F0E0FC4FF6FF71C0F60D018C4229D931
S31508002488B4F1016F38BF09211AD326E04FF00001CD
S3150800249816E04FF0010113E04FF0020110E04FF08B
S315080024A803010DE04FF004010AE04FF0050107E0CB
S315080024B84FF0060104E04FF0070101E04FF008016C
S315080024C801EB410346F27872C0F6000202EB83007C
S315080024D8007A10BD4FF0FF0010BD4FF0FF0010BD89
S315080024E82DE9F04105460068FFF742FFFF283BD073
S315080024F8FFF776FA4FF0F300FFF792FAFFF796FA26
S31508002508012818BF002404D1FFF780FA4FF0000409
S315080025182CE02F6804EB07082B195E6800F08AFC84
S3150800252840463146FFF7CAFA082815D1E059B0429D
S3150800253815D104F104042F6804EB07082A1956680C
S3150800254800F078FC40463146FFF7B8FA082810D05C
S3150800255802E04FF0010404E04FF0000401E04FF0F8
S315080025680004FFF753FA01E04FF000042046BDE8DF
S31508002578F081E359B342F2D104F10404B4F5007FBB
S31508002588C7D1E6E708B54FEAC1534FEAD3525AB955
S3150800259803688B420BD040F8041B4FF40072FFF710
S315080025A8B3FE4FF0010008BD4FF0000008BD4FF01C
S315080025B8010008BD38B504460D4640F21033C2F28C
S315080025C8000398420AD04FF40040C0F60000814242
S315080025D809D02046FFF784FF48B911E040F21454A1
S315080025E8C2F2000403E040F21034C2F200042046A6
S315080025F82946FFF7C7FF002814BF2046002038BD24
S315080026084FF0000038BD00BF2DE9F04704460D46D7
S3150800261816461F464FEA51294FEA49290368B3F176
S31508002628FF3F04D14946FFF7ADFF00283FD0206891
S31508002638484506D020464946FFF7BCFF0446002809
S3150800264839D021686D1A651905F1040540F2FF1895
S3150800265809F5007907F1FF3A0AF0010A00F0EAFBE2
S3150800266804F10402AB1A434536D92CE000F0E2FB24
S3150800267804F10400291A414507D920464946FFF7B7
S3150800268899FF0446D8B100F1040516F8012B05F898
S31508002698012B07F1FF3700F0CDFB04F10403E81A14
S315080026A8404542D938E04FF00100BDE8F0874FF0C1
S315080026B80000BDE8F0874FF00000BDE8F0874FF04E
S315080026C80000BDE8F08720464946FFF773FF044631
S315080026D80028F4D000F1040516F8010B05F8010BDB
S315080026E8013FE0D0BAF1000FC0D000F0A3FB04F117
S315080026F804016A1A424508D920464946FFF75AFF8F
S3150800270804460028DBD000F1040516F8013B05F855
S31508002718013B013FAAD1C6E720464946FFF74AFFCB
S3150800272804460028CBD000F1040516F8011B05F865
S31508002738011B013F9AD1B6E74FF0FF3340F2145216
S31508002748C2F20002136040F21030C2F200000360C1
S31508002758704700BF70B504460D461646FFF708FED3
S31508002768FF2823D004F1FF304019FFF701FEFF28A0
S315080027781FD04FEA54224FF40043C0F60003B3EBC8
S31508002788422F09D140F21030C2F2000021463246E3
S315080027982B46FFF739FF70BD40F21450C2F200000D
S315080027A8214632462B46FFF72FFF70BD4FF0000033
S315080027B870BD4FF0000070BD2DE9F04106460C4685
S315080027C8FFF7D6FD054606F1FF300019FFF7D0FDDD
S315080027D80446FF2D59D0FF285BD0854249D8012DDC
S315080027E84BD90B284DD8FFF7FBF84FF0F300FFF746
S315080027F817F9FFF71BF9012805D1FFF707F94FF075
S315080028080000BDE8F08146F24876C0F600064FF0AB
S315080028180207631B03F0010800F00CFB36F81500E5
S315080028283946FFF76BF9082837D008E000F002FBAD
S3150800283836F815003946FFF761F9082805D0FFF775
S31508002848E5F84FF00000BDE8F08105F1010505F04F
S31508002858FF0500F0EFFA36F815003946FFF74EF986
S31508002868082832D0EBE7FFF7D1F84FF00100BDE8AA
S31508002878F0814FF00000BDE8F0814FF00000BDE898
S31508002888F0814FF00000BDE8F0814FF00000BDE888
S31508002898F0814FF00000BDE8F08105F10105EDB2C1
S315080028A8AC42E0D34FFA88F10029BFD000F0C2FA4B
S315080028B836F815003946FFF721F90828BFD105F17A
S315080028C80105EDB2AC42B1D2CDE705F10105EDB28D
S315080028D8AC42ABD2C7E700BF00B583B040F21033AD
S315080028E8C2F200031868B0F1FF3F1ED040F2103359
S315080028F8C2F2000399685A688818D96840181A698C
S315080029088118586909189A698818DB69C118C1F1C4
S31508002918000002AA42F8040D48F28810C0F6000022
S315080029284FF00401FFF716FF01E04FF0010003B06E
S3150800293800BD00BF48F20402C0F600024FF4004387
S31508002948C0F6000310681968421848F20803C0F66A
S3150800295800031868111848F20C02C0F6000213683A
S31508002968C81848F21001C0F600010A68801848F22B
S315080029781403C0F600031968421848F21800C0F68E
S3150800298800000368D11848F28812C0F600021068D9
S315080029980B18D3F1010038BF0020704708B540F27C
S315080029A81033C2F200031868B0F1FF3F06D040F2B0
S315080029B81030C2F20000FFF793FD88B140F21451B7
S315080029C8C2F200010A68B2F1FF3F0CD040F2145077
S315080029D8C2F20000FFF784FD003018BF012008BDC9
S315080029E84FF0000008BD4FF0010008BD08B5FFF715
S315080029F8A3FE08BD08B5FFF7ADFE08BD08B5FFF785
S31508002A08DBFE08BD08B5FFF795FF08BD08B5FFF753
S31508002A1863FF10B1FFF7C2FF08BD4FF0000008BDFD
S31508002A284EF21003CEF200034FF000021A60704708
S31508002A3808B5FFF7F5FF4EF21003CEF2000349F288
S31508002A483F02C0F202025A604FF0000098604FF049
S31508002A580501196040F21873C2F20003186008BD30
S31508002A684EF21003CEF20003186810F4803F07D020
S31508002A7840F21871C2F200010A6802F101020A60FE
S31508002A88704700BF08B5FFF7EBFF40F21873C2F2AC
S31508002A980003186808BD00BF10B504464FF4A050D7
S31508002AA8C4F201004FF02001FFF716FB012809D1EF
S31508002AB84FF4A050C4F20100FFF708FB20704FF04E
S31508002AC8010010BD4FF0000010BD00BF38B5044620
S31508002AD84FF4A050C4F201004FF08001FFF7FCFA4A
S31508002AE8A8B14FF4A050C4F201002146FFF7E8FA4E
S31508002AF84FF4A054C4F201044FF080052046294635
S31508002B08FFF7EAFA0028F9D04FF0010038BD4FF070
S31508002B18000038BD10B584B04FF4614300934FF0F8
S31508002B280000ADF80400ADF80600ADF80800ADF8E9
S31508002B380C004FF00C01ADF80A104FF4A054C4F27B
S31508002B48010420466946FFF727FA20464FF0010197
S31508002B58FFF7A6FA04B010BD2DE9F84305460C465A
S31508002B68402907D946F2F070C0F600004FF0760102
S31508002B7800F0BCF82046FFF7A9FF012807D046F25F
S31508002B88F070C0F600004FF0790100F0AFF826465D
S31508002B9844B346F2F077C0F600074FF081084FF0C5
S31508002BA8000406F1FF3303F0010900F043F9285D34
S31508002BB8FFF78CFF012817D11AE000F03BF9285DCA
S31508002BC8FFF784FF012803D03846414600F08EF8FF
S31508002BD804F1010400F02EF9285DFFF777FF0128B4
S31508002BE820D123E0BDE8F8833846414600F07EF850
S31508002BF804F10104012EF5D90FFA89F00028DCD072
S31508002C0800F018F9285DFFF761FF012803D0384658
S31508002C18414600F06BF804F10104A1B2B142CCD3E5
S31508002C28BDE8F8833846414600F060F804F1010427
S31508002C38A2B2B242C1D3BDE8F88300BF10B50446B4
S31508002C4840F26173C2F200031878B0B940F21C70FA
S31508002C58C2F20000FFF720FF01283CD140F2617359
S31508002C68C2F200034FF0010018704FF0000040F25E
S31508002C786071C2F20001087010BD40F26071C2F2BC
S31508002C8800010A7802F1010240F21C73C2F200033D
S31508002C989818FFF701FF012820D140F26070C2F2A8
S31508002CA80000017801F10101CAB2027040F21C73F2
S31508002CB8C2F200031878904213D120460A49FFF752
S31508002CC823FB40F26171C2F200014FF000020A705C
S31508002CD84FF0010010BD4FF0000010BD4FF0000086
S31508002CE810BD4FF0000010BD1D07002008B540F2C2
S31508002CF86473C2F20003186040F26870C2F20000FA
S31508002D08016000F097F8FCE708B500F08DF801288F
S31508002D1820D000F05FFBE8B140F26C73C2F2000302
S31508002D281878012816D1FFF7ADFE40F27071C2F285
S31508002D3800010A6802F1320290420BD340F26C7322
S31508002D48C2F200034FF00000187000F04DFB08B9F6
S31508002D58FFF7C4FA08BD00BF08B540F26C73C2F2A3
S31508002D6800034FF001021A70FFF78CFE40F27071EB
S31508002D78C2F200010860FFF7C7FF08BD08B500F0F2
S31508002D8857F8FFF755FEFFF731FE00F00BFB00F08A
S31508002D980FF8FFF7E1FF08BD08B500F04BF8FFF795
S31508002DA85FFE00F07DFC00F01DF8FFF7ADFF08BDDB
S31508002DB800B583B04FF0FF038DF804304FF00000DC
S31508002DC88DF8050000F04EF8FFF7A4FE40F274717E
S31508002DD8C2F200010A78012A02D101A800F066F8B1
S31508002DE803B000BD08B540F27870C2F20000FFF7DC
S31508002DF825FF012805D140F27870C2F2000000F0DC
S31508002E0855F808BD704700BF08B5C9B2FFF7A4FE54
S31508002E1800F042F808BD00BF40F27473C2F200031E
S31508002E284FF001021A70704708B500F02BF808BD74
S31508002E38704700BF704700BF40F2B873C2F200037C
S31508002E484FF000025A70704740F2B873C2F2000396
S31508002E584FF0FE02DA7018714FF00200A3F844002A
S31508002E68704700BF40F2B873C2F200034FF0000281
S31508002E781A709A6483F84320A3F844209A705A7003
S31508002E88704700BF40F2B873C2F2000318780030E2
S31508002E9818BF0120704700BF40F2B873C2F200039A
S31508002EA84FF0000283F84320704700BF38B5044640
S31508002EB80378FF2B25D100F08DFA20B94FF01000C2
S31508002EC8FFF7C2FFC7E1FFF7B7FF40F2B873C2F2D0
S31508002ED800034FF001021A704FF0FF00D8704FF048
S31508002EE8100119714FF0000159714FF0400098719F
S31508002EF8D87119725A729A724FF00802A3F84420C8
S31508002F08A9E140F2B872C2F200021078012840F02E
S31508002F18BC81A3F1C903352B00F29981DFE813F0C8
S31508002F28FD009701970192019701970184011E01F7
S31508002F386A0154019701970197019701970197012B
S31508002F4897019701970197019701970197019701AB
S31508002F58970197019701970197019701970197019B
S31508002F68970197019701970197019701970197018B
S31508002F78970197018200540036007400970197015B
S31508002F889701B9009701D300D800EC0062783F2A68
S31508002F9804D94FF02200FFF757FF5CE140F2B875F5
S31508002FA8C2F2000505F10400A96CFFF7ADF94FF068
S31508002FB8FF00E8706178AB6CCA18AA64607800F1FB
S31508002FC80100A5F8440046E161783F2904D94FF085
S31508002FD82200FFF739FF3EE1616840F2B875C2F290
S31508002FE80005A96405F104006278FFF78DF94FF02A
S31508002FF8FF03EB706278A86C1118A964637803F16B
S315080030080103A5F8443026E140F2B870C2F2000080
S315080030184FF0FF01C170636883644FF00102A0F89E
S31508003028442018E140F2B870C2F200004FF0FF02DF
S31508003038C270836C6468C4B1E4186FEA030108199E
S3150800304800F0010213F8011BA34240F01F810EE0AD
S315080030581A4612F8010B09185B7853FA81F0C1B2BF
S3150800306802F10103A342F3D101E04FF0000140F257
S31508003078B873C2F20003C3F807104FF001021A71B9
S315080030884FF00001597199714FF00800A3F84400F0
S31508003098E1E040F2B870C2F200004FF0FF03C370D7
S315080030A846F67002C0F6000282644FF0000101710C
S315080030B8417181714FF00703C0F807304FF00802D5
S315080030C8A0F84420C7E04FF00000FFF7BDFEC2E0B5
S315080030D840F2B870C2F200004FF0FF01C1704FF01D
S315080030E800030371427842718371C37103724FF00A
S315080030F80601A0F84410AEE040F2B874C2F2000423
S315080031084FF000012170FFF797FE4FF0FF03E370B9
S315080031184FF00102A4F844209DE040F2B873C2F2C9
S315080031280003986C4FF03F0104F10102FFF762FCB7
S3150800313820B94FF03100FFF787FE8CE040F2B870EF
S31508003148C2F200004FF0FF01C170826C02F13F0223
S3150800315882644FF00103A0F844307CE063783E2B84
S3150800316804D94FF02200FFF76FFE74E040F2B870FA
S31508003178C2F200004FF0FF01C1704FF00102A0F83B
S315080031884420617841B9FFF741FC002863D14FF024
S315080031983100FFF759FE5EE040F2B873C2F2000349
S315080031A8986C04F10202FFF725FC20B94FF03100AC
S315080031B8FFF74AFE4FE040F2B870C2F200006178A5
S315080031C8826C8B18836446E040F2B873C2F2000337
S315080031D84FF0FF02DA704FF00000187158714FF07F
S315080031E840019971D871187258724FF00702A3F8FE
S315080031F8442030E040F2B873C2F20003986C616864
S31508003208FFF7FCFB20B94FF03100FFF71DFE22E05F
S3150800321840F2B870C2F200004FF0FF01C1704FF0DB
S315080032280102A0F8442016E0FFF79EF840F2B870AD
S31508003238C2F200004FF0FF01C1704FF00102A0F87A
S31508003248442008E04FF03100FFF7FEFD03E04FF099
S315080032582000FFF7F9FD40F2B873C2F2000393F8AD
S315080032684310012903D14FF01000FFF7EDFD40F296
S31508003278B873C2F200034FF0010083F8430003F164
S315080032880300B3F84410FFF7BFFD38BD002A3FF422
S31508003298DFAE13F8010B0918C9B2A3427FF4D8AEFA
S315080032A8E5E600BF30B402464CF6CD44CCF6CC442D
S315080032B801F10101A4FB0223DA08F9D14FF0000550
S315080032C801F8015902464CF6CD45CCF6CC450846D8
S315080032D8A5FB02434FEAD30303EB8304A2EB44029C
S315080032E802F1300201F801291A46002BEFD130BC49
S315080032F8704700BF38B50546007803F075F9C0B2BF
S31508003308A0F13004E4B2162C20D8A0F13A02D1B2C2
S3150800331806291ED9092C84BFA0F13704E4B26878B7
S3150800332803F062F9C0B2A0F13003D9B2162913D84E
S31508003338A0F13A02D3B2062B11D9092984BFA0F104
S315080033483701C9B201EB0414E0B238BD4FF00000EA
S3150800335838BD4FF0000038BD4FF0000038BD4FF0BB
S31508003368000038BD08B500F00F03092802D903F193
S31508003378370008BD03F1300003F036F9C0B208BDBE
S3150800338838B505460C464FEA1010FFF7EBFF2070D4
S3150800339805F00F00FFF7E6FF60704FF00003A37013
S315080033A8204638BD08B54FF0000040F64403C2F27F
S315080033B80003187040F65001C2F2000102F0A6FB9D
S315080033C838B146F67800C0F600004FF07C01FFF7E2
S315080033D88DFC08BD40F64403C2F200031878D0F104
S315080033E8010038BF0020704708B5FFF71DFD012802
S315080033F80FD040F64403C2F20003187860B9FEF706
S3150800340871FE01280BD140F64401C2F2000108708A
S3150800341808BD4FF0000008BD4FF0000008BD4FF08A
S31508003428000008BD10B50446007803F0DDF85328F7
S315080034380DD1607803F0D0F860B1607831280CD0E7
S3150800344832280DD0332814BF0320022010BD4FF0B0
S31508003458030010BD4FF0030010BD4FF0000010BD6B
S315080034684FF0010010BD00BFF8B5044600F1020090
S31508003478FFF740FF0646054604F1040400F0010775
S315080034882046FFF737FF3018C6B205F1FF318DB26F
S3150800349804F10204012D21D815E02046FFF72AFF7A
S315080034A83018C6B205F1FF3504F10204ADB220465C
S315080034B8FFF720FF3118CEB205F1FF3295B204F1B5
S315080034C80204012DE9D82046FFF714FF6FEA060320
S315080034D8DEB2864214BF00200120F8BD3FB2002F95
S315080034E8DBD02046FFF706FF3218D6B205F1FF33C0
S315080034F89DB204F10204012DCFD8E4E72DE9F04185
S3150800350804461546884601B138B946F67800C0F625
S31508003518000040F23621FFF7E9FB2046FFF782FF55
S315080035280646032800F0B0802046FFF79DFF0028CE
S3150800353800F0AD80012E34D01EB1022E40F0AA80CC
S3150800354865E004F10200FFF7D5FE074604F104001A
S31508003558FFF7D0FE4FEA0026C8F8006004F1060017
S31508003568FFF7C8FE3118C8F8001004F10804A7F1D7
S315080035780307BFB2002D00F08F800FFA87F8B8F15D
S31508003588000F40F389804FF000062046FFF7B2FE89
S31508003598A85504F1020406F10106B6B24645F4DB5D
S315080035A87AE004F10200FFF7A5FE074604F10400D5
S315080035B8FFF7A0FE4FEA0046C8F8006004F10600C7
S315080035C8FFF798FE06EB0026C8F8006004F1080025
S315080035D8FFF790FE3218C8F8002004F10A04A7F18C
S315080035E80407BFB2002D57D00FFA87F8B8F1000FB5
S315080035F852DD4FF000062046FFF77CFEA85504F179
S31508003608020406F10106B6B24645F4DB44E004F1C5
S315080036180200FFF76FFE074604F10400FFF76AFE8B
S315080036284FEA0066C8F8006004F10600FFF762FE74
S3150800363806EB0046C8F8006004F10800FFF75AFED2
S3150800364806EB0026C8F8006004F10A00FFF752FEE8
S315080036583018C8F8000004F10C04A7F10507BFB232
S31508003668D5B10FFA87F8B8F1000F15DD4FF0000647
S315080036782046FFF73FFEA85504F1020406F10106A5
S31508003688B6B24645F4DB07E04FF0000704E04FF60C
S31508003698FF7701E04FF0000738B2BDE8F08100BFB8
S315080036A870B540F64403C2F200031878002800F003
S315080036B84D82012843D1FEF73FFD46F6EC00C0F6D9
S315080036C80000FEF787FD46F61010C0F60000FEF764
S315080036D881FDFEF72BFD0146C6484FF0010202F0B0
S315080036E82FFA50B146F63810C0F60000FEF772FDFC
S315080036F84FF00100FEF75EFD70BD46F64010C0F6B5
S315080037080000FEF767FD46F64810C0F60000FEF70B
S3150800371861FD46F66C10C0F60000FEF75BFD40F644
S315080037284803C2F200034FF000021A605A6040F6D6
S315080037384400C2F200004FF00201017070BD022871
S3150800374840F0088140F65004C2F2000440F6A8404A
S31508003758C2F200004FF4807104F50D7202F07EFE85
S3150800376894F93A12002915DA46F63810C0F6000018
S31508003778FEF730FD4FF00200FEF71CFD04F50D704C
S3150800378802F0F0FC40F64400C2F200004FF00001D7
S31508003798017070BD18B340F6A846C2F20006304656
S315080037A806F5C0714FF00002FFF7A8FE0646B0F10D
S315080037B8FF3F14D146F63810C0F60000FEF70AFD9A
S315080037C84FF00300FEF7F6FC8A4802F0CBFC40F6F9
S315080037D84403C2F200034FF000021A7070BD32B2F9
S315080037E8002A2CDD40F64803C2F20003586868B977
S315080037F840F64801C2F2000140F6A843C2F20003A7
S31508003808D3F88001086036B24E6018E040F6A84141
S31508003818C2F20001D1F8802140F64803C2F200033B
S3150800382819688A4204D240F64803C2F200031A60AD
S3150800383800FA86F040F64802C2F20002506040F6E6
S315080038485001C2F20001D1F83C22D1F840329A421E
S3150800385840F07C8167484FF0000102F08FFCA0B168
S3150800386846F63810C0F60000FEF7B4FC4FF0040020
S31508003878FEF7A0FC5F4802F075FC40F64400C2F269
S3150800388800004FF00001017070BD46F64010C0F602
S315080038980000FEF79FFC46F69C10C0F60000FEF7EF
S315080038A899FC40F64804C2F2000440F60405C2F240
S315080038B8000560682946FFF7F5FC2846FEF78AFCE6
S315080038C846F6A810C0F60000FEF784FCE0782946FC
S315080038D8FFF756FDA07805F10201FFF751FD60785C
S315080038E805F10401FFF74CFD207805F10601FFF7FD
S315080038F847FD2846FEF76EFC46F64C20C0F6000043
S31508003908FEF768FC20686168FFF778F8A0B946F6FC
S315080039183810C0F60000FEF75DFC4FF00500FEF70C
S3150800392849FC344802F01EFC40F64403C2F2000380
S315080039384FF000021A7070BD46F64010C0F6000037
S31508003948FEF748FC40F64400C2F200004FF00301B7
S31508003958017070BD032840F0F98040F65004C2F2A1
S31508003968000440F6A840C2F200004FF4807104F53E
S315080039780D7202F073FD94F93A12002915DA46F623
S31508003988C410C0F60000FEF725FC4FF00200FEF74B
S3150800399811FC04F50D7002F0E5FB40F64403C2F28B
S315080039A800034FF00000187070BD28B340F6A8420F
S315080039B8C2F20002104602F5C07102F58072FFF7DE
S315080039C89DFD0546B0F1FF3F16D146F6E810C0F64C
S315080039D80000FEF7FFFB4FF00300FEF7EBFB054878
S315080039E802F0C0FB40F64401C2F200014FF00002A3
S315080039F80A7070BD840A00202BB2002B5EDD46F6DD
S31508003A080C20C0F60000FEF7E5FB2EB240F60404CB
S31508003A18C2F2000430462146FFF744FC2046FEF76A
S31508003A28D9FB46F61C20C0F60000FEF7D3FB40F685
S31508003A38A845C2F2000595F883012146FFF7A0FCC0
S31508003A4895F8820104F10201FFF79AFC95F88101BD
S31508003A5804F10401FFF794FC95F8800104F10601C6
S31508003A68FFF78EFC2046FEF7B5FB46F64C20C0F657
S31508003A780000FEF7AFFBD5F88001314605F58072E0
S31508003A88FEF7B8FFA0B946F63810C0F60000FEF7EC
S31508003A98A1FB4FF00600FEF78DFB2D4802F062FBEE
S31508003AA840F64403C2F200034FF00000187070BDD8
S31508003AB846F64010C0F60000FEF78CFB40F65000AC
S31508003AC8C2F20000D0F83C12D0F8402291423DD10B
S31508003AD846F63420C0F60000FEF77CFBFEF796FF94
S31508003AE8A0B946F63810C0F60000FEF773FB4FF08B
S31508003AF80700FEF75FFB164802F034FB40F6440160
S31508003B08C2F200014FF000020A7070BD46F6401076
S31508003B18C0F60000FEF75EFB46F65020C0F6000029
S31508003B28FEF758FB0A4802F01DFB46F66820C0F661
S31508003B380000FEF74FFB40F64403C2F200034FF0BD
S31508003B4800001870FEF714FBFEF7C8FB70BD00BF2F
S31508003B58840A002010B4E2B182186FEA0004131927
S31508003B6803F0010401F1FF3111F8013F00F8013BA8
S31508003B78904210D10DE001F101044978034603F893
S31508003B88011B04F101016478447003F101009042B5
S31508003B98F1D110BC7047002CEDD011F8013F00F8A0
S31508003BA8013B9042E7D1F4E792B182186FEA000325
S31508003BB8D31803F0010300F8011B904209D1704796
S31508003BC8034603F8011B417003F101009042F7D13F
S31508003BD87047002BF4D000F8011B9042F0D17047CB
S31508003BE8037833B18B4204D010F8013F0BB18B42EE
S31508003BF8FAD11846704700BFCA7E8B7E43EA02236D
S31508003C080078032805D1487D097D41EA002243EA60
S31508003C1802431846704700BF8176C1F30723C37667
S31508003C284FEA114101754FEA11224275704700BFE4
S31508003C3803784FEAC31242EA53014378CA18D1B245
S31508003C484FEAC11343EA5101827852FA81F3D9B28D
S31508003C584FEAC11242EA5103C17851FA83F2D3B244
S31508003C684FEAC31141EA5303027952FA83F1CBB2F8
S31508003C784FEAC31242EA5301437953FA81F2D1B2A1
S31508003C884FEAC11343EA5101827952FA81F3D9B24C
S31508003C984FEAC11242EA5103C17951FA83F2D3B203
S31508003CA84FEAC31141EA5303027A52FA83F1CBB2B7
S31508003CB84FEAC31242EA5301437A53FA81F2D1B260
S31508003CC84FEAC11343EA5101807A50FA81F2D0B219
S31508003CD8704700BF08B5024688B1036893B11978DA
S31508003CE899B1D8889288904212D15878FDF714FD70
S31508003CF800F00103002B14BF0320002008BD4FF075
S31508003D08090008BD4FF0090008BD4FF0090008BDB5
S31508003D184FF0090008BD00BF10B504460A464078AA
S31508003D2804F134014FF00103FDF710FD00283ED1D8
S31508003D3894F8332294F8323243EA022001B24AF65A
S31508003D485522CFF6FF72914234D194F86D0094F853
S31508003D586C304FEA034141EA006294F86A0042EA85
S31508003D68000394F86B1043EA012222F07F4044F2DC
S31508003D784613C0F2540398421FD094F8891094F851
S31508003D8888204FEA024040EA016194F8863041EA01
S31508003D98030294F8870042EA002121F07F4244F2A0
S31508003DA84613C0F25403D01A18BF012010BD4FF0AD
S31508003DB8030010BD4FF0020010BD4FF0000010BD03
S31508003DC82DE9F041154603681C78A4F13004092C3E
S31508003DD800F2E5815A783A2A40F0E18103F10203B4
S31508003DE803604FF000030B60002C40F08C8141F211
S31508003DF83004C2F200042468002C00F088810C60A4
S31508003E08217889B16078FDF787FC10F0010F0BD18E
S31508003E18002D00F0808100F00401C8B2002814BF04
S31508003E280A200020BDE8F0814FF00000207060707D
S31508003E38FDF754FC10F0010F40F071812DB100F028
S31508003E480402D0B2002840F06E8120464FF00001E7
S31508003E58FFF762FF012819D194F8F631002B00F014
S31508003E68668194F8FD5194F8FC114FEA014242EA3A
S31508003E78056094F8FA3140EA030194F8FB5141EADF
S31508003E88052520462946FFF747FF01E04FF00005BC
S31508003E98032800F05081002840F0518194F840200A
S31508003EA894F83F0040EA022319B2B1F5007F40F0C2
S31508003EB84A8194F84B2094F84A0050EA02210FD117
S31508003EC894F85B1094F85A304FEA034242EA0160C4
S31508003ED894F8581040EA010394F8592043EA022155
S31508003EE8E16194F84420E27002F1FF30C3B2012B75
S31508003EF800F22D8194F84130A370002B00F02B8135
S31508003F0803F1FF30184240F02A8194F8466094F885
S31508003F18450040EA0626B0B2208116F00F0F40F099
S31508003F28228194F8487094F8476056EA07260ED115
S31508003F3894F8577094F856604FEA064646EA0767B3
S31508003F4894F854603E4394F8557046EA072694F860
S31508003F5843C094F8427057EA0C2700F0088102FB20
S31508003F6801FC07EB101262449642C0F00481B61AA7
S31508003F78B6FBF3F3002B00F0028140F6F576B34260
S31508003F888CBF022601264FF6F578434500F20B81C9
S31508003F9803F10203A3612562EF1967625219E26207
S31508003FA8032E15D1002840F0EE8094F8630094F8A3
S31508003FB862204FEA024242EA006094F8602002430F
S31508003FC894F8610042EA0022A2624FEA830011E0EF
S31508003FD8002800F0DC806744A762022E02D14FEA67
S31508003FE8430007E04FF0030000FB03F203F0010368
S31508003FF803EB520000F2FF13B1EB532FC0F0CB804E
S315080040084FF0FF3121614FF00000E060032E6CD1BC
S31508004018607194F8652094F8643043EA02216A18B6
S315080040286261607804F134014FF00103FDF78EFBF5
S3150800403800285AD194F8330294F8322242EA002327
S3150800404819B24AF65520CFF6FF7081424DD194F839
S31508004058372094F836304FEA034141EA026094F86B
S31508004068342040EA020394F8351043EA012045F261
S315080040785222C4F26112904237D194F81B1294F86E
S315080040881A324FEA034040EA016294F8181242EAE3
S31508004098010394F8190243EA002247F27221C6F28C
S315080040A841118A4221D194F8230294F822324FEA20
S315080040B8034242EA006194F8200241EA000394F8B0
S315080040C8212243EA0221E16094F81F0294F81E327D
S315080040D84FEA034242EA006194F81C0241EA0003E7
S315080040E894F81D2243EA0221216126703348038881
S315080040F803F101039AB20280E2804FF000002063C0
S315080041082071BDE8F0814FF00B00BDE8F0814FF053
S315080041180C00BDE8F0814FF00000BDE8F0814FF0D3
S315080041280300BDE8F0814FF00A00BDE8F0814FF0C2
S315080041380D00BDE8F0814FF00100BDE8F0814FF0B1
S315080041480D00BDE8F0814FF00D00BDE8F0814FF095
S315080041580D00BDE8F0814FF00D00BDE8F0814FF085
S315080041680D00BDE8F0814FF00D00BDE8F0814FF075
S315080041780D00BDE8F0814FF00D00BDE8F0814FF065
S315080041880D00BDE8F0814FF00D00BDE8F0814FF055
S315080041980D00BDE8F0814FF00D00BDE8F0814FF045
S315080041A80000086023E603F10203A3612562EF19FC
S315080041B867625619E6624FF00306F3E62C100020EC
S315080041C82DE9F0410C4601F109020369002B00F0BC
S315080041D8E28043691E7B1978202900F08A80052920
S315080041E814BF0A46E52206F0080505F0FF0135B1B1
S315080041F8A2F14105EDB2192D9CBF2032D2B26272E6
S3150800420804F10A025D78202D73D0052D08BFE5252F
S3150800421831B1A5F14102D2B2192A9CBF2035EDB2B7
S31508004228A57204F10B029D78202D62D0052D08BFD2
S31508004238E52531B1A5F14102D2B2192A9CBF20352C
S31508004248EDB2E57204F10C02DD78202D51D0052D6A
S3150800425808BFE52531B1A5F14102D2B2192A9CBF9A
S315080042682035EDB2257304F10D021D79202D40D0B5
S31508004278052D08BFE52531B1A5F14102D2B2192AA3
S315080042889CBF2035EDB2657304F10E025D79202DC9
S315080042982FD0052D08BFE52531B1A5F14102D2B2C7
S315080042A8192A9CBF2035EDB2A57304F10F029D7932
S315080042B8202D1ED0052D08BFE52531B1A5F14102EF
S315080042C8D2B2192A9CBF2035EDB2E57304F1100263
S315080042D8DD79202D0DD0052D08BFE52531B1A5F1CD
S315080042E84101CAB2192A9CBF2035EDB2257404F1DA
S315080042F811021D7A202D36D015464FF02E0105F8E5
S31508004308011B197A20292DD006F0100606F0FF059C
S3150800431836B1A1F14106F6B2192E9CBF2031C9B2B1
S31508004328517002F10206597A20290DD035B1A1F14A
S315080043384106F6B2192E9CBF2031C9B2917002F116
S315080043480306997A202901D132460CE035B1A1F144
S315080043584105EEB2192E9CBF2031C9B2D17002F1BF
S31508004368040200E02A46D97A2172DD7F9E7F4FEA49
S31508004378064141EA05661D7F2E43597F46EA01260E
S3150800438826605D7E197E41EA0526A680D97D9B7D35
S3150800439843EA0126E6804FF000011170A6698EB33C
S315080043A8E2697AB30569E5B1018C4FF6FF7399425C
S315080043B81AD0C7693888D0B14FF00005A8464146D3
S315080043C802F0B4F80146A8B1E06900F1FF32AA4242
S315080043D813D9715505F1010537F8020F0028EED1F2
S315080043E80DE04FF000050AE04FF0000507E04FF032
S315080043F8000504E04FF0000501E04FF000054FF016
S3150800440800037355BDE8F0812DE9F843044603799E
S31508004418002B40D0076B00F13405407829463A4608
S315080044284FF00103FDF7CCF9002838D14FF000000A
S315080044382071616A8F4236D3E2698B189F4236D259
S31508004448E678012E37D94FF0010806EA0809BF1899
S31508004458607829463A464346FDF7B2F906F1FF362B
S3150800446846452CD113E0E269BF18607829463A46D2
S315080044784346FDF7A5F9E369FF18607829463A46E1
S315080044884346FDF79DF9A6F10206012EEBD14FF03A
S315080044980000BDE8F8834FF00000BDE8F8834FF048
S315080044A80100BDE8F8834FF00000BDE8F8834FF037
S315080044B80000BDE8F8834FF00000BDE8F883B9F1BD
S315080044C8000FD0D0E1697F18607829463A464346F6
S315080044D8FDF776F906F1FF36012EC4D1D7E700BFF6
S315080044E838B504460D46036B8B420DD0FFF78CFF93
S315080044F868B9607804F134012A464FF00103FDF7DC
S3150800450825F938B9256338BD4FF0000038BD4FF096
S31508004518010038BD4FF0010038BD00BF70B504462C
S31508004528FFF772FF034600285FD12378032B53D180
S315080045386079002850D04FF00005256304F1340649
S31508004548304629464FF40072FFF72EFB4FF0550107
S3150800455884F832124FF0AA0284F833224FF0520335
S3150800456884F8343084F835304FF0610084F8360022
S315080045784FF0410284F837204FF0720184F8181278
S3150800458884F8191284F81A2284F81B02236984F815
S315080045981C32C3F3072084F81D024FEA134284F835
S315080045A81E224FEA136184F81F12E36884F8203242
S315080045B8C3F3072084F821024FEA134284F822221B
S315080045C84FEA136184F823126078314662694FF01E
S315080045D80103FDF7F5F8657160784FF000010A46A2
S315080045E8FDF72CF9031C18BF0123184670BD00BF38
S315080045F8A1F102018369A3F10203994204D28278E0
S31508004608C06A02FB010070474FF00000704700BF00
S31508004618F8B505460C4601296DD9836999426DD2C4
S315080046280078022832D0032845D0012869D101EB41
S315080046385106696A284601EB5621FFF751FF0028FB
S3150800464862D14FEAC6524FEAD257EB1993F834703B
S3150800465806F10106696A284601EB5621FFF740FF6D
S31508004668002854D14FEAC6564FEAD656AD1995F8DA
S31508004678340047EA002214F0010F02D04FEA12105C
S31508004688F8BD4FEA02534FEA1350F8BD6A6A28463E
S3150800469802EB1121FFF724FF00283BD14FEA0464F7
S315080046A84FEAD4502B1893F834102C1894F8352060
S315080046B841EA0220F8BD696A284601EBD411FFF7DA
S315080046C80FFF002829D14FEA44644FEAD4516B18E2
S315080046D893F8360093F837204FEA026444EA004212
S315080046E893F8353042EA03206C1894F834100843D6
S315080046F820F07040F8BD4FF00100F8BD4FF00100FA
S31508004708F8BD4FF0FF30F8BD4FF0FF30F8BD4FF059
S31508004718FF30F8BD4FF0FF30F8BD4FF0FF30F8BD59
S3150800472870B504460D46E180816801293CD00368C6
S315080047389A6991423BD279B91878032801D1996ABE
S3150800474851B94FF00000E0601A89AA4232D99B6A2B
S3150800475803EB151121611CE09E784FEA0616B5424F
S3150800476810D32068FFF754FF0146B0F1FF3F24D065
S31508004778012825D923689A69904224D2AD1BADB27F
S31508004788AE42EED9E1602068FFF732FF00EB15115B
S31508004798216105F00F05206800EB451202F1340285
S315080047A862614FF0000070BD4FF0020070BD4FF017
S315080047B8020070BD4FF0020070BD4FF0010070BDD9
S315080047C84FF0020070BD4FF0020070BDF8B50546FF
S315080047D80C461646012940F28C808369994280F076
S315080047E88B800078022845D0032858D001287AD12A
S315080047F801EB5107696A284601EB5721FFF770FE56
S315080048080346002871D14FEAC7524FEAD25314F02B
S31508004818010409D0E91891F8342002F00F00F1B222
S3150800482840EA0112D0B200E0F0B2EB1883F834007F
S3150800483807F101074FF001002871696A284601EB5C
S315080048485721FFF74DFE034600284ED14FEAC757B2
S315080048584FEAD75014B1C6F3071607E02A1892F894
S31508004868341021F00F07C6F303263E432F1887F89E
S3150800487834603AE06B6A284603EB1121FFF730FEED
S31508004888034690BB4FEA04644FEAD452A91881F844
S3150800489834600C46C6F3072681F8356025E06B6A4E
S315080048A8284603EBD111FFF71BFE0346E8B94FEA82
S315080048B844644FEAD4502A1892F837104FEA01612F
S315080048C82C1801F07040064384F83460C6F30721B3
S315080048D882F835104FEA164082F836004FEA16660F
S315080048E882F8376001E04FF002034FF001002871A3
S315080048F804E04FF0020301E04FF002031846F8BD42
S315080049082DE9F0410546884631B9C66876B1836906
S315080049189E4228BF01260BE0FFF77AFE03460128C8
S3150800492845D9AA6990424CD3464601E04FF001069C
S3150800493834464FF0020704F10104A869844202D3F9
S31508004948012E37D93C4628462146FFF761FE03461D
S3150800495838B1B0F1FF3F34D0012832D0B442EAD199
S315080049682BE02646284621466FF07042FFF72EFFB1
S315080049780146B0B9B8F1000F06D028464146224686
S31508004988FFF724FF014660B9EE602A69B2F1FF3FD6
S3150800499816D002F1FF3028614FF0010169712346EC
S315080049A80FE0012914BF01234FF0FF3309E04FF048
S315080049B8010306E04FF0000303E04FF0000300E0B0
S315080049C823461846BDE8F0812DE9F84304460E4605
S315080049D8C58805F10105ADB2002D70D00369002B15
S315080049E871D015F00F075FD103F101030361C168A0
S315080049F821B903681989A94269D955E000688278F6
S31508004A0802F1FF3313EA15134ED1FFF701FE80466C
S31508004A18012860D9B0F1FF3F61D0206881698845CF
S31508004A283BD3002E5FD0E168FFF76AFF804600286F
S31508004A385DD001285FD0B0F1FF3F60D02068FFF74E
S31508004A48E3FC00285FD1206800F134004FF000012C
S31508004A584FF40072FFF7A8F8266830464146FFF774
S31508004A68C7FD30634FF000064FF001090EE080F8E5
S31508004A7804902068FFF7C8FC002848D12068026B14
S31508004A8802F10102026306F10106F6B2206882788D
S31508004A98B242ECD8036B991B0163C4F80C802068F2
S31508004AA84146FFF7A5FD2061E580206800EB47121F
S31508004AB802F1340262614FF00000BDE8F8834FF056
S31508004AC80400BDE8F8834FF00400BDE8F8834FF00A
S31508004AD80400BDE8F8834FF00200BDE8F8834FF0FC
S31508004AE80100BDE8F8834FF00400BDE8F8834FF0ED
S31508004AF80700BDE8F8834FF00200BDE8F8834FF0D9
S31508004B080100BDE8F8834FF00100BDE8F8834FF0CF
S31508004B180100BDE8F88300BF2DE9F04F83B00446CD
S31508004B284FF00001FFF7FCFD0746002840F02C82ED
S31508004B384FF0FF0BD846DA464FF00009206821697E
S31508004B48FFF7CEFC0746002840F01E8265692E78D6
S31508004B58002E00F00B82EB7A03F03F02E52E00F0F8
S31508004B68E18103F00800C1B219B10F2A40F0DC81CF
S31508004B7802E00F2A40F09881E769002F00F0ED81DE
S31508004B8806F04003DAB232B195F80DB006F0BF0662
S31508004B98E188218404E0B04518BFD04640F0DD819D
S31508004BA8687B0090584540F0C1812B7823F0400275
S31508004BB802F1FF3101EB410001EB80030193AA786A
S31508004BC8697841EA022001F0EDFC80460198FE2842
S31508004BD800F2D68100F1010B37F8100001F0E2FC6B
S31508004BE8804540F0CD812A79EB7843EA0220B8F16E
S31508004BF8000F04D14FF6FF71884211D0C0E101F0C9
S31508004C08D1FC8046BBF1FE0F00F2BA8137F81B00CB
S31508004C18019A02F1020B01F0C5FC804540F0B0810B
S31508004C28A8796B7943EA0020B8F1000F04D14FF64A
S31508004C38FF71884210D0A3E101F0B4FC8046BBF1AD
S31508004C48FE0F00F29D8137F81B000BF1010B01F0EE
S31508004C58A9FC804540F094812A7AE87940EA02203E
S31508004C68B8F1000F04D14FF6FF73984210D087E1C8
S31508004C7801F098FC8046BBF1FE0F00F2818137F8F7
S31508004C881B000BF1010B01F08DFC804540F0788183
S31508004C98A97A6A7A42EA0120B8F1000F04D14FF6D8
S31508004CA8FF73984210D06BE101F07CFC8046BBF19B
S31508004CB8FE0F00F2658137F81B000BF1010B01F0B6
S31508004CC871FC804540F05C81E87BA97B41EA0020BD
S31508004CD8B8F1000F04D14FF6FF72904210D04FE199
S31508004CE801F060FC8046BBF1FE0F00F2498137F8F7
S31508004CF81B000BF1010B01F055FC804540F0408183
S31508004D08687C2B7C43EA0020B8F1000F04D14FF6E3
S31508004D18FF71884210D033E101F044FC8046BBF1AC
S31508004D28FE0F00F22D8137F81B000BF1010B01F07D
S31508004D3839FC804540F02481EA7CA87C40EA0220B8
S31508004D48B8F1000F04D14FF6FF73984210D017E157
S31508004D5801F028FC8046BBF1FE0F00F2118137F8F6
S31508004D681B000BF1010B01F01DFC804540F0088182
S31508004D78697D2A7D42EA0120B8F1000F04D14FF671
S31508004D88FF73984210D0FBE001F00CFC8046BBF19B
S31508004D98FE0F00F2F58037F81B000BF1010B01F046
S31508004DA801FC804540F0EC80E87DA97D41EA0020B9
S31508004DB8B8F1000F04D14FF6FF72904210D0DFE029
S31508004DC801F0F0FB8046BBF1FE0F00F2D98037F8F8
S31508004DD81B000BF1010B01F0E5FB804540F0D08084
S31508004DE8687E2B7E43EA0020B8F1000F04D14FF6FF
S31508004DF8FF71884210D0C3E001F0D4FB8046BBF1AE
S31508004E08FE0F00F2BD8037F81B000BF1010B01F00D
S31508004E18C9FB804540F0B4806A7F287F40EA0220B3
S31508004E28B8F1000F04D14FF6FF73984210D0A7E0E7
S31508004E3801F0B8FB8046BBF1FE0F00F2A18037F8F7
S31508004E481B000BF1010B01F0ADFB804540F0988083
S31508004E58E97FAA7F42EA0120B8F1000F10D001F0D5
S31508004E68A1FB8046BBF1FE0F00F28A800BF1010018
S31508004E78019037F81B0001F095FB804505D07FE0C7
S31508004E884FF6FF77B84274D07AE02B7803F04001E2
S31508004E98CAB2002A6DD0B8F1000F6AD0019837F85F
S31508004EA81070002F65D06BE0B8F1000F04D12846C2
S31508004EB8FEF7BEFE584567D04FF0FF332384A06936
S31508004EC8C27A12F0010F33D129780378994231D181
S31508004ED86978427891422FD1AB7881788B422DD167
S31508004EE8EB78C27893422BD129790379994229D14B
S31508004EF869794279914227D1AB7981798B4225D153
S31508004F08EB79C279934223D1297A037A994221D136
S31508004F18697A427A91421FD1A97A807A814233D036
S31508004F28D0461AE0D04618E0D04616E0D04614E037
S31508004F38D04612E0D04610E0D0460EE0D0460CE047
S31508004F48D0460AE0D04608E0D04606E0D04604E057
S31508004F58D04602E0D04600E0D04620464946FFF74C
S31508004F6833FD074600283FF4E9AD0DE04FF0040786
S31508004F780AE006F1FF365FFA86F8DDF800B0ECE7D6
S31508004F88DDF800B0D046E8E7384603B0BDE8F08F4C
S31508004F982DE9F04F87B001908B460B782F2B01D05F
S31508004FA85C2B01D10BF1010B4FF0000001998860C9
S31508004FB89BF800201F2A0AD808464FF00001FFF779
S31508004FC8AFFB02464FF0000301994B6198E146F69C
S31508004FD89424C0F60004039446F6A026C0F60006F4
S31508004FE8049646F6A823C0F6000305935E461BF802
S31508004FF8010B2F28FAD05C28F8D00199CA690292C1
S3150800500830781F2840F256812F2800F045815C2801
S3150800501800F047811746A7F1020735464FF0010405
S31508005028A34613E02F2B00F040815C2B00F03D814E
S31508005038B2F5807F00F0598192461446594601F028
S3150800504875FA8046002840F08D814EE1594601F0F0
S315080050586DFA8046002800F048817F2806D803980C
S315080050684146FEF7BDFD002840F03F8107F10209D9
S31508005078A7F8028015F8013F184604F101021F2B0C
S31508005088D0D81BE1002C00F0308104F1FF3000F085
S315080050980101029B03EB440232F8020D202840F076
S315080050A8478148E132F8023D202B01D02E2B08D142
S315080050B804F1FF30041E32F8021D202940F04B8106
S315080050C84CE12746002C00F01081029A02EB4408AE
S315080050D84FF0000522F81450019B98694FF02001FB
S315080050E84FF00B02FEF760FD029AA2F1020201E0F8
S315080050F805F1010532F8020F2028F9D02E28F7D035
S31508005108002D00F0E08046F00306DCE004F1FF30ED
S31508005118044628B94FF008094FF00008C24607E0C8
S31508005128A8F1020737F8021C2E2940F0F780F1E7A4
S31508005138029B33F8157005F10105002F5AD0202F68
S3150800514804D02E2F05D1AC4200F0D28046F00306D3
S31508005158EEE7C84502D2AC4217D1C1E0B9F10B0F48
S3150800516803D146F00306504647E0AC4203D046F062
S315080051780306A54240D84FEA8A0A5FFA8AFA2546FC
S315080051884FF00B094FF00808D2E77F2F0FD938469A
S315080051984FF0000101F0CAF90746002800F0AD8073
S315080051A80598C11911F8807C46F0020627B10498BB
S315080051B83946FEF715FD20B146F003064FF05F079E
S315080051C811E0A7F1410293B2192B02D84AF0020A54
S315080051D809E0A7F1610081B2192904D84AF0010A41
S315080051E8A7F12007BFB2019A936903F8087008F176
S315080051F801089DE7504600E0504601998B691A78E0
S31508005208E52A04BF05221A70B9F1080F04BF800001
S315080052185FFA80FA0AF00C000C2803D00AF003019A
S31508005228032901D146F0020606F00203DAB252B99A
S315080052380AF0030ABAF1010F08BF46F01006042857
S3150800524808BF46F0080601988169CE72FFF764FC24
S31508005258019B9A69D37A024640B1042850D103F0D3
S315080052680403D8B2002808BF052249E003F0040061
S31508005278C1B2002944D1019A5169CB7A03F01000CA
S31508005288C2B232B1019C2068FEF7B6FC019EB06036
S31508005298ACE64FF0050233E04FF000044FF0010288
S315080052A803E04FF000044FF0010206EB020B4FF043
S315080052B80006E7E64FF000044FF0010206EB020B82
S315080052C84FF00406DEE607F1FF37029931F8172092
S315080052D82E2A3FF41FAF14F0010F7FF417AF13E01F
S315080052E8B9F10B0F7FF447AF3BE74FF0060207E02B
S315080052F8B9F10B0F7FF43FAF33E746F002065BE7D9
S31508005308104607B0BDE8F08F04F1FF34A8F102088B
S3150800531838F8023C2E2B7FF4F9AEFBE600F1FF3491
S31508005328A7F1020838F8022C2E2A7FF4EFAEF1E628
S315080053382E287FF4C6AE013CD7D000293FF4B2AE7A
S3150800534832F8021D202902D02E297FF4BAAE013C74
S315080053587FF4A8AEC9E72E297FF4B3AE441E7FF4BE
S31508005368A1AEC2E77F2805D803984146FEF738FC60
S315080053780028BAD109F10207A9F8028015F8011F11
S31508005388084604F101021F2998D92F298DD05C29CE
S315080053988BD00AF1010459E62DE9F0410446C5887F
S315080053A8018C4FF6FF73994208BF2946FFF7B8F9EB
S315080053B80346E0B94FF0E5074FF001064FF000083D
S315080053C820682169FFF78CF8034668B9626917707F
S315080053D820680671E188A94209D220464146FFF7A6
S315080053E8F3FA03460028EBD0042B08BF0223184615
S315080053F8BDE8F0812DE9F84F044689464FF0FF0AC3
S3150800540856464FF00405D0464FF000074FF6FF7B87
S315080054183AE12068FFF764F80546002840F0398124
S3150800542860690378002B00F04081C27AE52B00F00A
S315080054381E812E2B00F01D8102F03F02082A14BF98
S3150800544800210121494540F016810F2A40F00681BE
S3150800545803F04001CDB235B190F80DA003F0BF03B3
S31508005468E688268404E09E4218BF464640F0068130
S31508005478417B514540F00181E669027802F03F0513
S3150800548805F1FF3202EB420E02EB8E0E8578427862
S3150800549842EA0525BEF1FE0F00F2048126F81E50E1
S315080054A80EF1010290F804A090F803C04CEA0A2A03
S315080054B815B9DA4508D0F5E0FE2A00F2F38026F891
S315080054C812A00EF10202554690F806C090F805E0BB
S315080054D84EEA0C2A15B9DA4508D0E3E0FE2A00F2A6
S315080054E8E18026F812A002F10102554690F808C094
S315080054F890F807E04EEA0C2A15B9DA4508D0D1E043
S31508005508FE2A00F2CF8026F812A002F101025546BB
S3150800551890F80AC090F809E04EEA0C2A15B9DA4557
S3150800552808D0BFE0FE2A00F2BD8026F812A002F1D4
S315080055380102554690F80FC090F80EE04EEA0C2A7C
S3150800554815B9DA4508D0ADE0FE2A00F2AB8026F890
S3150800555812A002F10102554690F811C090F810E021
S315080055684EEA0C2A15B9DA4508D09BE0FE2A00F25D
S31508005578998026F812A002F10102554690F813C040
S3150800558890F812E04EEA0C2A15B9DA4508D089E0EF
S31508005598FE2A00F2878026F812A002F10102554673
S315080055A890F815C090F814E04EEA0C2A15B9DA45B1
S315080055B807D077E0FE2A75D826F812A002F101026C
S315080055C8554690F817C090F816E04EEA0C2A15B911
S315080055D8DA4507D066E0FE2A64D826F812A002F152
S315080055E80102554690F819C090F818E04EEA0C2AB8
S315080055F815B9DA4507D055E0FE2A53D826F812A079
S3150800560802F10102554690F81DC090F81CE04EEAD2
S315080056180C2A15B9DA4507D044E0FE2A42D826F8F6
S3150800562812A002F10102554690F81FC090F81EE034
S315080056384EEA0C2A35B1FE2A34D826F812A002F109
S31508005648010201E0DA452DD1007800F04005E8B2FC
S3150800565818B3FE2A26D826F812701EE01EB9FEF7D9
S31508005668E7FA504524D04FF6FF70208420E04646D6
S3150800567804E0464602E0464600E0464620463946E5
S31508005688FFF7A2F9054620B9216900297FF4C1AEBA
S3150800569875B14FF0000121610AE003F1FF33DEB26C
S315080056A88A46EBE78A464646E8E74FF00405F0E7F8
S315080056B82846BDE8F88F00BF2DE9F04104460E4696
S315080056C8012926D98369994226D24FF000074FF057
S315080056D8010820463146FEF79BFF0546F8B1012822
S315080056E820D0B0F1FF3F20D0204631463A46FFF792
S315080056F86DF80146D8B92069B0F1FF3F04D000F12A
S315080057080100206184F805802E46A269AA42E0D8DD
S315080057180DE04FF002010AE04FF0020107E04FF0F2
S31508005728000104E04FF0020101E04FF001010846CC
S31508005738BDE8F08170B582B0054616461C464FF09E
S315080057480B02FEF707FA052C0DD9A6F102024FEA55
S31508005758540343EAC43432F8020F10FA84F18CB2BF
S315080057685688002EF3D14FF0070204F00F0000F117
S315080057783003392B88BF00F137030DF8023002F1E0
S31508005788FF322409F1D1164602A988184FF07E037C
S3150800579800F8083C92B12C78202C12D029464FF0F4
S315080057A8000312F0010F56D003F101000346B04278
S315080057B809D011F8014F202C54D104E04FF000030A
S315080057C801E04FF000034FF02000C3F1070101F094
S315080057D80104072A19D811E0072A06D802ACA11825
S315080057E811F8081C02F1010200E00146E95403F128
S315080057F80103072A28D820E002B070BD02AEB11806
S3150800580811F8081C02F1010200E00146E95403F107
S315080058180103072BF0D8002CDED0072A06D802ACDD
S31508005828A11811F8081C02F1010200E00146E95422
S3150800583803F10103072BCFD9DEE702AEB11811F839
S31508005848081C02F1010200E00146E95403F10103CC
S31508005858072BC1D9D0E703F1010311F8010F202856
S31508005868A2D1B0E700F1010311F8010F20289BD156
S31508005878A9E700BF2DE9F04F87B004468769C669CE
S3150800588803A839464FF00C02FEF764F99DF817305D
S3150800589813F0010F2FD04FF00000F872E0614FF0B7
S315080058A80105384603A932462B46FFF743FF20462B
S315080058B8FFF732F9814698B905F10105ADB23846C0
S315080058C803A932462B46FFF735FF2046FFF724F98A
S315080058D88146002800F0038102E04FF00709FAE044
S315080058E8642D00F0DB80B9F1040F40F0F4809DF8D0
S315080058F81710F972E6619DF8172002F00207FBB245
S31508005908DBB1308848B14FF0000303F101039BB2BD
S3150800591836F813100029F8D101E04FF0000303F117
S3150800592819034EF64F42C4F6C46282FB03174FEAC0
S31508005938E370C0EBA7039FB201E04FF001072046CA
S315080059484FF00001FEF7ECFE8146002840F0C380C0
S315080059584FF00005A8464FF0010620682169FEF7B2
S31508005968BFFD8146002840F0B68061690A78E52AB5
S3150800597800D022B905F10105AF4201D191E04546AB
S3150800598820463146FFF720F881460028E5D0A2E0F0
S31508005998E088C31B204699B2FEF7C2FE8146002856
S315080059A840F09980A069FEF743F901904FF0000886
S315080059B84FF6FF7546F62836C0F6000620682169B0
S315080059C8FEF78EFD8146002840F08580D4F81C90A5
S315080059D861695FFA87FB019A4A734FF00F00C8722C
S315080059E881F80C8081F81A8081F81B800BF1FF3347
S315080059F803EB430203EB82004FF0010243464FF0E4
S31508005A08FF0A02E02B4602F10102AB424ED039F8F2
S31508005A18103000F1010006EB020C1CF801EC01F845
S31508005A280E308E444FEA132C8EF801C0002B48D04E
S31508005A380C2AE8D9AB4202D039F8100018B947F051
S31508005A48400B5FFA8BFB81F800B022684FF0010122
S31508005A58117120464146FEF7B7FF814600283AD11C
S31508005A6807F1FF37BFB2002FA8D12DE060694FF0C4
S31508005A7800014FF02002FEF797F86069A1694FF018
S31508005A880B02FEF767F86369A069C27A02F0180183
S31508005A98197323684FF0010018711CE04FF00709C5
S31508005AA819E007F1FF37BFB277B171E706EB020EC7
S31508005AB81EF801CC01F80CA001EB0C0E8EF801A01B
S31508005AC8B6E70C2A9ED9BAE720682169FEF708FDC9
S31508005AD881460028CAD0484607B0BDE8F08F05F1C8
S31508005AE80105ADB2384603A932462B46FFF722FE12
S31508005AF82046FFF711F8814600287FF4F1AE05F134
S31508005B080105ADB2642D7FF4CCAEE6E6A0B941F244
S31508005B183003C2F20003186810B14FF00002027091
S31508005B2811B14FF000030B7041F23000C2F20000C9
S31508005B3801604FF0000070474FF00B00704700BF38
S31508005B482DE9F0438FB0019116460546002800F066
S31508005B58A5804FF00003036001A805A902F01E02FC
S31508005B68FEF72EF90446002840F0B78006F01F080D
S31508005B7802A80B9040F62C61C2F200010C9105A808
S31508005B880199FFF705FA0A9F0146002840F08F8019
S31508005B98002F40F0868088E059B1042940F09280A9
S31508005BA805A8FFF767FE48F008080A9F50B104469B
S31508005BB893E0FB7A13F0110F7ED106F00402D6B2F1
S31508005BC8002E7CD108F00800C6B2002E41D0FBF79B
S31508005BD86FFEB873C0F30723FB734FEA10423A7493
S31508005BE84FEA106179744FF00006FE723E777E77A9
S31508005BF8BE77FE7705983946FDF7FEFF8146384693
S31508005C083146FEF709F805984FF001030371B9F113
S31508005C18000F1ED0066B4946FFF74EFD002853D1E4
S31508005C28059809F1FF31C1603146FEF759FC01466E
S31508005C380DE0FB7A03F01002D0B2002846D106F030
S31508005C480206F6B22EB113F0010F42D101E000297F
S31508005C5842D108F00800C6B20EB148F02008059EE1
S31508005C68336BEB612F6285F8068030463946FDF7B7
S31508005C78C3FF2861FA7FB97F4FEA014040EA026309
S31508005C883A7F1343797F43EA0120E8604FF000031F
S31508005C98AB60AB612E60F288AA801EE04FF009045B
S31508005CA81BE016F01C0F84D1C3E74FF0060116F067
S31508005CB81C0F7FF471AFCAE74FF007040DE04FF0E9
S31508005CC808040AE00C4608E0044606E04FF0040417
S31508005CD803E04FF0070400E00C4620460FB0BDE885
S31508005CE8F08300BF2DE9F04F83B0044688469146F5
S31508005CF81E464FF000033360FDF7ECFF0746002801
S31508005D0840F0D080A07910F0800F40F0C68010F0DF
S31508005D18010F00F0C580E568A1686D1AA94538BF66
S31508005D284D46002D00F0BE8004F12402009201972A
S31508005D38A7684FEAC7534FEAD350002840F08D802A
S31508005D48206890F802A00AF1FF3101EA572212F0FA
S31508005D58FF0A19D10FB9206902E06169FEF758FCF4
S31508005D68012806D8A77967F07F00A0714FF00207C7
S31508005D7898E0B0F1FF3F06D1A37963F07F02A271DC
S31508005D884FF001078EE06061276838466169FEF7BB
S31508005D982FFC814630B9A07960F07F01A1714FF0D8
S31508005DA802077FE000EB0A095FEA552B29D0BB7882
S31508005DB80BEB0A029A4288BFCAEB030B787841466E
S31508005DC84A465FFA8BF3FBF7C1FC30B1A27962F059
S31508005DD87F07A7714FF0010764E0A77907F040002D
S31508005DE8C1B259B1A369C9EB0302934506D908EBB1
S31508005DF8422000994FF40072FDF7ACFE4FEA4B2B90
S31508005E083CE0A2694A4526D0A37903F04000C1B20E
S31508005E1889B1787800994FF00103FBF7D1FC30B1C6
S31508005E28A07960F07F01A1714FF001073AE0A279E5
S31508005E3822F04007A7712368587800994A464FF018
S31508005E480103FBF783FC30B1A77967F07F03A371D9
S31508005E584FF0010726E0C4F81890A0684FEAC05129
S31508005E684FEAD152C2F5007B5D4538BFAB46A1184B
S31508005E78404601F124015A46FDF76CFED844A76846
S31508005E8807EB0B00A060316801EB0B033360B5EB39
S31508005E980B057FF44DAF019F04E04FF0020701E0C0
S31508005EA84FF00707384603B0BDE8F08F2DE9F04FE5
S31508005EB883B00446884615461E464FF000033360ED
S31508005EC8FDF708FF0746002840F0EE80A07910F095
S31508005ED8800F40F0E48000F00201CAB2002A00F000
S31508005EE8E180E368DD4280F0D080002D00F0CD80A7
S31508005EF804F1240000900197A7684FEAC7514FEAB2
S31508005F08D152002A40F09C80206890F802B00BF124
S31508005F18FF3303EA572111F0FF0B24D147B9276944
S31508005F286FB94FF00001FEF7EBFC0746206103E066
S31508005F386169FEF7E5FC0746002F00F0A580012FEA
S31508005F4806D1A77967F07F00A0714FF00207ABE08A
S31508005F58B7F1FF3F06D1A27962F07F03A3714FF02C
S31508005F680107A1E06761A07900F04002D3B29BB1AE
S31508005F78216848780099A2694FF00103FBF720FCCD
S31508005F8830B1A07960F07F01A1714FF001078BE06D
S31508005F98A77927F04000A071276838466169FEF797
S31508005FA827FB814630B9A37963F07F07A7714FF0BD
S31508005FB8020779E000EB0B095FEA552A28D0B97879
S31508005FC80AEB0B028A4288BFCBEB010A787841466E
S31508005FD84A465FFA8AF3FBF7F3FB30B1A17961F019
S31508005FE87F02A2714FF001075EE0A369C9EB0307B8
S31508005FF8BA450AD9009808EB47214FF40072FDF70D
S31508006008A9FDA07920F04001A1714FEA4A2A2CE09F
S31508006018A2694A4512D0A168E36899420ED27878EF
S3150800602800994A464FF00103FBF790FB30B1A07977
S3150800603860F07F07A7714FF0010735E0C4F818909C
S31508006048A0684FEAC0574FEAD752C2F5007A5545B5
S3150800605838BFAA46A01800F1240041465246FDF763
S3150800606879FDA17941F04003A371D044A26802EBF7
S315080060780A03A360376807EB0A003060B5EB0A0520
S315080060887FF43AAF019F00E0019FA168E268914258
S3150800609888BFE160A37943F02000A07104E04FF0BF
S315080060A8020701E04FF00707384603B0BDE8F08F4E
S315080060B838B50446FDF70EFE0346002850D1A279E6
S315080060C802F02001C8B200284AD002F04003DAB22A
S315080060D872B1214651F8240B4078A2694FF00103A2
S315080060E8FBF76EFB002839D1A17921F04003A3718B
S315080060F82068E169FEF7F4F9034688BB256AEA7A57
S3150800610842F02000E872E1682977A3894FEA13224A
S315080061186A77E089A877E17BE97728462169FDF758
S315080061287BFDFBF7C5FBA875C0F30723EB754FEA9C
S3150800613810422A764FEA106068764FF00001A97473
S31508006148E974A37923F02002A27120684FF00101AF
S3150800615801712068FEF7E2F9034601E04FF00103F2
S31508006168184638BD10B50446FFF7A2FF034610B90E
S315080061784FF000022260184610BD00BFF8B5044665
S315080061880D46FDF7A7FD0746002840F0D380A379FA
S3150800619813F0800F40F0CC80E268AA4205D203F0DB
S315080061A80200C1B2002908BF1546A2684FF00003CD
S315080061B8A360002D00F0BE80206886784FEA462640
S315080061C882B102F1FF3205F1FF31B1FBF6F1B2FBFC
S315080061D8F6F3994206D3C6F100031A40A260AD1A2F
S315080061E8616919E02169B1B9FEF78AFB01460128F8
S315080061F806D1A27962F07F01A1714FF0020799E0F2
S31508006208B0F1FF3F06D1A77967F07F00A0714FF07C
S3150800621801078FE020616161002946D0B5422ED971
S31508006228A07900F00202D3B22BB12068FEF768FB0A
S31508006238014620B922E02068FEF7EAF90146B1F1DD
S31508006248FF3F06D1A27962F07F03A3714FF00107D9
S3150800625870E0012903D920688269914206D3A77993
S3150800626867F07F01A1714FF0020763E06161A368D7
S315080062789819A060AD1BAE42D2D300E03546A06897
S315080062884219A2604FEAC5534FEAD35080B1206835
S31508006298FEF7AEF930B9A07960F07F07A7714FF01D
S315080062A8020747E000EB552504E04FF0000501E03A
S315080062B84FF00005A2684FEAC2534FEAD35068B3B5
S315080062C8A269AA422AD0A17901F04003D8B298B1A6
S315080062D8214651F8243B58784FF00103FBF770FA2A
S315080062E830B1A27962F07F01A1714FF0010721E070
S315080062F8A27922F04001A171214651F8240B407871
S315080063082A464FF00103FBF721FA30B1A77967F05F
S315080063187F03A3714FF001070CE0A561A368E26843
S31508006328934207D9E360A17941F02000A07101E002
S315080063384FF002073846F8BD30B58FB00EAB43F8B4
S31508006348340D0D46184605A94FF00002FDF738FD2D
S315080063580446A8B902A80B9040F62C61C2F20001BF
S315080063680C9105A80199FEF713FE044640B90A9A46
S3150800637822B105A82946FDF723FF01E04FF00604D8
S3150800638820460FB030BD00BF30B599B018AB43F8FA
S315080063985C0D18460FA94FF00102FDF711FD0246DC
S315080063A8002857D103A8159040F62C61C2F20001BF
S315080063B816910FA80199FEF7EBFD0246002849D168
S315080063C8149959B3CC7A14F0010F2AD12CE0012D6F
S315080063D834D906A80FA94FF02402FDF7BBFB089588
S315080063E806A84FF00201FEF79BF90246002831D1AC
S315080063F806A84FF00001FEF7FDFF024640B3042841
S315080064081FD027E02DB10F982946FFF755F9024600
S3150800641800BB0F98FEF782F802461BE04FF006020B
S3150800642818E04FF0070215E00F98FDF7E5FB05465B
S3150800643804F01004E4B2002CC9D102E04FF00202BD
S3150800644808E00FA8FEF7A8FF02460028DAD001E000
S315080064584FF00702104619B030BD00BF2DE9F047C6
S3150800646882B08246914604464FF0000501F1FF378F
S315080064784FF0010814E0484601A942466B46FFF763
S3150800648831FC009B012B0ED19DF804000D2808D07D
S31508006498307004F10104264605F101050A2802D0E0
S315080064A82646AF42E7DC4FF0000131708D4214BF33
S315080064B85046084602B0BDE8F08700BF30B583B03D
S315080064C804460D460A2803D14FF00D00FFF7F6FFDC
S315080064D802A901F8084D284669464FF0010201ABA2
S315080064E8FFF7E4FC0198012814BF4FF0FF3001209C
S315080064F803B030BD70B505460E46007870B14FF04A
S3150800650800043146FFF7DAFFB0F1FF3F09D004F17E
S31508006518010415F8010F0028F3D104E04FF0000430
S3150800652801E04FF0FF34204670BD00BF7F282DD903
S3150800653811B9C7280BD121E0FF2825D8A0F180007A
S3150800654846F61852C0F6000232F8100070474FF0A7
S31508006558010346F61852C0F6000232F8021F8142B5
S3150800656815D10DE032F8021F814209D003F1010363
S315080065789BB232F8021F81420DD101E04FF00003A9
S3150800658803F18000C0B270474FF00000704703F16E
S3150800659801039BB2E6E703F101039BB2802BE1D125
S315080065A8EEE700BF61280ED046F63831C0F600017E
S315080065B84FF0000202F1010231F8023F5BB1834253
S315080065C8F8D113B970474FF0000246F61860C0F6BE
S315080065D8000030F812007047A0F1300009288CBF77
S315080065E800200120704700BFA0F16103D9B219291C
S315080065F898BF2038704700BF844640EA010313F065
S31508006608030F40F01080242AC0F00D802DE9F00F02
S31508006618B1E8F80FA0E8F80FA2F12402242ABFF47B
S31508006628F7AFBDE8F00F002A00F0078011F8013B24
S3150800663800F8013B013A7FF4F9AF6046704700BF9E
S3150800664838B504460D4600F019F841F23403C2F28B
S3150800665800031D6044F0800441F23800C2F20000CD
S315080066680460024611680029FCD100F009F841F2D5
S315080066783403C2F20003186838BD00BF704700BF6C
S30908006688704700BF8A
S3150800668C2F64656D6F70726F675F6F6C696D657877
S3150800669C5F73746D3332653430372E7372656300ED
S315080066AC2F626F6F746C6F672E747874000000001D
S315080066BC433A2F576F726B2F736F667477617265D7
S315080066CC2F4F70656E424C542F5461726765742F48
S315080066DC44656D6F2F41524D434D345F53544D33C2
S315080066EC325F4F6C696D65785F53544D3332453460
S315080066FC30375F43726F7373776F726B732F426F9A
S3150800670C6F742F6964652F2E2E2F2E2E2F2E2E2F5B
S3150800671C2E2E2F536F757263652F41524D434D3490
S3150800672C5F53544D33322F43726F7373776F726B9B
S3150800673C732F766563746F72732E630000000800FE
S3150800674C10001800200028003000380040004800CF
S3150800675C500058008000880090009800A000A800FF
S3150800676CB000B800C000C800D000D80000800008EF
S3150800677C004000000200000000C0000800400000B5
S3150800678C03000000000001080000010004000000DE
S3150800679C00000208000002000500000000000408C2
S315080067AC00000200060000000000060800000200B7
S315080067BC070000000000080800000200080000009E
S315080067CC00000A08000002000900000000000C087E
S315080067DC000002000A00000000000E08000002007B
S315080067EC0B000000433A2F576F726B2F736F66744A
S315080067FC776172652F4F70656E424C542F546172D7
S3150800680C6765742F44656D6F2F41524D434D345F48
S3150800681C53544D33325F4F6C696D65785F53544DE5
S3150800682C3332453430375F43726F7373776F726BDD
S3150800683C732F426F6F742F6964652F2E2E2F2E2E91
S3150800684C2F2E2E2F2E2E2F536F757263652F4152B6
S3150800685C4D434D345F53544D33322F756172742E3C
S3150800686C630000004F70656E424C5400433A2F5734
S3150800687C6F726B2F736F6674776172652F4F7065C5
S3150800688C6E424C542F5461726765742F44656D6F54
S3150800689C2F41524D434D345F53544D33325F4F6C39
S315080068AC696D65785F53544D3332453430375F43E1
S315080068BC726F7373776F726B732F426F6F742F6966
S315080068CC64652F2E2E2F2E2E2F2E2E2F2E2E2F5337
S315080068DC6F757263652F66696C652E630000000020
S315080068EC4669726D7761726520757064617465208E
S315080068FC7265717565737420646574656374656413
S3150800690C0A0D00004F70656E696E67206669726DB8
S3150800691C776172652066696C6520666F7220726590
S3150800692C6164696E672E2E2E000000004552524F88
S3150800693C520A0D004F4B0A0D000000005374617289
S3150800694C74696E67207468652070726F6772616D02
S3150800695C6D696E672073657175656E63650A0D00E2
S3150800696C50617273696E67206669726D77617265BC
S3150800697C2066696C6520746F206F627461696E207D
S3150800698C65726173652073697A652E2E2E00000078
S3150800699C45726173696E6720000000002062797485
S315080069AC65732066726F6D206D656D6F72792061E7
S315080069BC742030780000000052656164696E6720A7
S315080069CC6C696E652066726F6D2066696C652E2E15
S315080069DC2E4552524F520A0D00000000496E766140
S315080069EC6C696420636865636B73756D20666F7577
S315080069FC6E642E2E2E4552524F520A0D0000000080
S31508006A0C50726F6772616D6D696E672000000000C9
S31508006A1C20627974657320746F206D656D6F727959
S31508006A2C206174203078000057726974696E67208B
S31508006A3C70726F6772616D20636865636B73756DD1
S31508006A4C2E2E2E00436C6F73696E67206669726D05
S31508006A5C776172652066696C650A0D004669726D08
S31508006A6C77617265207570646174652073756363EC
S31508006A7C65737366756C6C7920636F6D706C657471
S31508006A8C65640A0D00000000222A3A3C3E3F7C7FD2
S31508006A9C000000002B2C3B3D5B5D0000809A90416A
S31508006AAC8E418F804545454949498E8F9092924F24
S31508006ABC994F555559999A9B9C9D9E9F41494F555F
S31508006ACCA5A5A6A7A8A9AAABAC21AEAFB0B1B2B37F
S31508006ADCB4B5B6B7B8B9BABBBCBDBEBFC0C1C2C3E4
S31508006AECC4C5C6C7C8C9CACBCCCDCECFD0D1D2D3D4
S31508006AFCD4D5D6D7D8D9DADBDCDDDEDFE0E1E2E3C4
S31508006B0CE4E5E6E7E8E9EAEBECEDEEEFF0F1F2F3B3
S31508006B1CF4F5F6F7F8F9FAFBFCFDFEFF0103050799
S31508006B2C090E10121416181C1E00000061006200D3
S31508006B3C63006400650066006700680069006A0007
S31508006B4C6B006C006D006E006F00700071007200B7
S31508006B5C73007400750076007700780079007A0067
S31508006B6CA100A200A300A500AC00AF00E000E10064
S31508006B7CE200E300E400E500E600E700E800E900CF
S31508006B8CEA00EB00EC00ED00EE00EF00F000F1007F
S31508006B9CF200F300F400F500F600F800F900FA002C
S31508006BACFB00FC00FD00FE00FF00010103010501CE
S31508006BBC070109010B010D010F0111011301150143
S31508006BCC170119011B011D011F01210123012501B3
S31508006BDC270129012B012D012F0131013301350123
S31508006BEC37013A013C013E0140014201440146018C
S31508006BFC48014B014D014F015101530155015701F4
S31508006C0C59015B015D015F01610163016501670162
S31508006C1C69016B016D016F017101730175017701D2
S31508006C2C7A017C017E019201B103B203B303B4036A
S31508006C3CB503B603B703B803B903BA03BB03BC035E
S31508006C4CBD03BE03BF03C003C103C303C403C5030B
S31508006C5CC603C703C803C903CA0330043104320484
S31508006C6C33043404350436043704380439043A0436
S31508006C7C3B043C043D043E043F04400441044204E6
S31508006C8C43044404450446044704480449044A0496
S31508006C9C4B044C044D044E044F0451045204530443
S31508006CAC5404550456045704580459045A045B04EE
S31508006CBC5C045E045F0470217121722173217421B6
S31508006CCC752176217721782179217A217B217C21DE
S31508006CDC7D217E217F2141FF42FF43FF44FF45FF73
S31508006CEC46FF47FF48FF49FF4AFF4BFF4CFF4DFF46
S31508006CFC4EFF4FFF50FF51FF52FF53FF54FF55FFF6
S31508006D0C56FF57FF58FF59FF5AFF0000C700FC00F3
S31508006D1CE900E200E400E000E500E700EA00EB0029
S31508006D2CE800EF00EE00EC00C400C500C900E60060
S31508006D3CC600F400F600F200FB00F900FF00D600CE
S31508006D4CDC00A200A300A500A7209201E100ED003B
S31508006D5CF300FA00F100D100AA00BA00BF00102314
S31508006D6CAC00BD00BC00A100AB00BB009125922570
S31508006D7C9325022524256125622556255525632547
S31508006D8C512557255D255C255B25102514253425AD
S31508006D9C2C251C2500253C255E255F255A255425C2
S31508006DAC69256625602550256C2567256825642583
S31508006DBC652559255825522553256B256A251825E9
S31508006DCC0C25882584258C2590258025B103DF0084
S31508006DDC9303C003A303C303B500C403A603980314
S31508006DECA903B4031E22C603B50329226122B100E6
S31508006DFC6522642220232123F7004822B000192299
S31508006E0CB7001A227F20B200A025A000410042003C
S31508006E1C43004400450046004700480049004A0024
S31508006E2C4B004C004D004E004F00500051005200D4
S31508006E3C53005400550056005700580059005A0084
S31508006E4C2100E0FFE1FFE5FFE2FFE3FFC000C10020
S31508006E5CC200C300C400C500C600C700C800C900EC
S31508006E6CCA00CB00CC00CD00CE00CF00D000D1009C
S31508006E7CD200D300D400D500D600D800D900DA0049
S31508006E8CDB00DC00DD00DE007801000102010401F4
S31508006E9C060108010A010C010E0110011201140168
S31508006EAC160118011A011C011E01200122012401D8
S31508006EBC260128012A012C012E0130013201340148
S31508006ECC360139013B013D013F01410143014501B1
S31508006EDC47014A014C014E01500152015401560119
S31508006EEC58015A015C015E01600162016401660188
S31508006EFC68016A016C016E017001720174017601F8
S31508006F0C79017B017D01910191039203930394030B
S31508006F1C950396039703980399039A039B039C037B
S31508006F2C9D039E039F03A003A103A303A403A50328
S31508006F3CA603A703A803A903AA03100411041204A1
S31508006F4C13041404150416041704180419041A0453
S31508006F5C1B041C041D041E041F0420042104220403
S31508006F6C23042404250426042704280429042A04B3
S31508006F7C2B042C042D042E042F04010402040304F0
S31508006F8C0404050406040704080409040A040B048B
S31508006F9C0C040E040F046021612162216321642113
S31508006FAC652166216721682169216A216B216C217B
S31508006FBC6D216E216F2121FF22FF23FF24FF25FF60
S31508006FCC26FF27FF28FF29FF2AFF2BFF2CFF2DFF63
S31508006FDC2EFF2FFF30FF31FF32FF33FF34FF35FF13
S31108006FEC36FF37FF38FF39FF3AFF000078
S31508006FF8010000000100000000000000010203046F
S30D0800700801020304060708094A
S70508000217D9
